
 Start         Length     Name                   Class
 0001:00000000 00018000H .text                   CODE
 0002:00000000 00000674H .data                   DATA
 0002:00000674 00000A15H .bss                    BSS


Detailed map of segments

 0001:00000000 0000528F C=CODE     S=.text    G=(none)   M=System   ACBP=A9
 0001:00005290 000001CC C=CODE     S=.text    G=(none)   M=SysInit  ACBP=A9
 0001:0000545C 00000038 C=CODE     S=.text    G=(none)   M=Types    ACBP=A9
 0001:00005494 000001D8 C=CODE     S=.text    G=(none)   M=Windows  ACBP=A9
 0001:0000566C 00000038 C=CODE     S=.text    G=(none)   M=Messages ACBP=A9
 0001:000056A4 000002C8 C=CODE     S=.text    G=(none)   M=SysConst ACBP=A9
 0001:0000596C 000042A0 C=CODE     S=.text    G=(none)   M=SysUtils ACBP=A9
 0001:00009C0C 00000098 C=CODE     S=.text    G=(none)   M=VarUtils ACBP=A9
 0001:00009CA4 00004264 C=CODE     S=.text    G=(none)   M=Variants ACBP=A9
 0001:0000DF08 000000E8 C=CODE     S=.text    G=(none)   M=RTLConsts ACBP=A9
 0001:0000DFF0 00000DCC C=CODE     S=.text    G=(none)   M=TypInfo  ACBP=A9
 0001:0000EDBC 00000038 C=CODE     S=.text    G=(none)   M=ActiveX  ACBP=A9
 0001:0000EDF4 00008C42 C=CODE     S=.text    G=(none)   M=Classes  ACBP=A9
 0001:00017A38 000005C5 C=CODE     S=.text    G=(none)   M=pluginexample ACBP=A9
 0002:00000000 0000008C C=DATA     S=.data    G=DGROUP   M=System   ACBP=A9
 0002:0000008C 00000028 C=DATA     S=.data    G=DGROUP   M=SysInit  ACBP=A9
 0002:000000B4 0000020C C=DATA     S=.data    G=DGROUP   M=SysUtils ACBP=A9
 0002:000002C0 00000108 C=DATA     S=.data    G=DGROUP   M=VarUtils ACBP=A9
 0002:000003C8 0000008E C=DATA     S=.data    G=DGROUP   M=Variants ACBP=A9
 0002:00000458 0000000C C=DATA     S=.data    G=DGROUP   M=TypInfo  ACBP=A9
 0002:00000464 0000003C C=DATA     S=.data    G=DGROUP   M=Classes  ACBP=A9
 0002:00001000 00000704 C=BSS      S=.bss     G=DGROUP   M=System   ACBP=A9
 0002:00001704 0000001C C=BSS      S=.bss     G=DGROUP   M=SysInit  ACBP=A9
 0002:00001720 00000004 C=BSS      S=.bss     G=DGROUP   M=Types    ACBP=A9
 0002:00001724 00000004 C=BSS      S=.bss     G=DGROUP   M=Windows  ACBP=A9
 0002:00001728 00000004 C=BSS      S=.bss     G=DGROUP   M=Messages ACBP=A9
 0002:0000172C 00000004 C=BSS      S=.bss     G=DGROUP   M=SysConst ACBP=A9
 0002:00001730 00000120 C=BSS      S=.bss     G=DGROUP   M=SysUtils ACBP=A9
 0002:00001850 00000004 C=BSS      S=.bss     G=DGROUP   M=VarUtils ACBP=A9
 0002:00001854 00000184 C=BSS      S=.bss     G=DGROUP   M=Variants ACBP=A9
 0002:000019D8 00000004 C=BSS      S=.bss     G=DGROUP   M=RTLConsts ACBP=A9
 0002:000019DC 00000004 C=BSS      S=.bss     G=DGROUP   M=TypInfo  ACBP=A9
 0002:000019E0 00000004 C=BSS      S=.bss     G=DGROUP   M=ActiveX  ACBP=A9
 0002:000019E4 00000030 C=BSS      S=.bss     G=DGROUP   M=Classes  ACBP=A9


  Address         Publics by Name

 0002:0000172C       .1
 0002:000019D8       .1
 0002:00001720       .1
 0002:00001850       .1
 0002:00001718       .1
 0002:00001728       .1
 0002:00001874       .3
 0002:000019E0       .3
 0002:00001724       .3
 0002:000019E8       .35
 0002:000015B4       .5
 0002:000019DC       .6
 0002:00001840       .94
 0001:00001884       @AbstractError
 0001:000026C8       @AfterConstruction
 0001:00001C14       @AStrCmp
 0001:000026D8       @BeforeDestruction
 0001:00002520       @CallDynaInst
 0001:00002670       @ClassCreate
 0001:000026C0       @ClassDestroy
 0001:00001BBC       @Close
 0001:00003CC8       @CopyArray
 0001:00003BAC       @CopyRecord
 0001:00003F38       @DispCallByIDError
 0001:00002B54       @DoneExcept
 0001:00004674       @DynArrayAsg
 0001:00004638       @DynArrayClear
 0001:00004524       @DynArrayCopy
 0001:00004544       @DynArrayCopyRange
 0001:00004364       @DynArrayHigh
 0001:0000435C       @DynArrayLength
 0001:00004518       @DynArraySetLength
 0001:00002C3C       @ExceptionHandler
 0001:00001C84       @FillChar
 0001:00003BA0       @Finalize
 0001:00003AB4       @FinalizeArray
 0001:00003A80       @FinalizeRecord
 0001:00001BB0       @Flush
 0001:0000227C       @FpuInit
 0001:000021B8       @FpuMaskInit
 0001:000016E8       @FreeMem
 0001:000016C8       @GetMem
 0001:00005390       @GetTls
 0001:000030E8       @Halt
 0001:00003010       @Halt0
 0001:000027EC       @HandleAnyException
 0001:00002AA0       @HandleFinally
 0001:00002918       @HandleOnException
 0001:00002ED4       @InitImports
 0001:000053DC       @InitLib
 0001:00002EAC       @InitResStringImports
 0001:00004CDC       @IntfClear
 0001:00004CF4       @IntfCopy
 0001:000024CC       @IsClass
 0001:00002188       @isNECWindows
 0001:000035A0       @LStrAddRef
 0001:00003124       @LStrArrayClr
 0001:00003154       @LStrAsg
 0001:000033C0       @LStrCat
 0001:00003404       @LStrCat3
 0001:00003478       @LStrCatN
 0001:00003100       @LStrClr
 0001:000034FC       @LStrCmp
 0001:00003610       @LStrCopy
 0001:00003650       @LStrDelete
 0001:00003368       @LStrFromArray
 0001:000032E0       @LStrFromChar
 0001:000032F0       @LStrFromPChar
 0001:000031F0       @LStrFromPCharLen
 0001:00003320       @LStrFromPWChar
 0001:00003254       @LStrFromPWCharLen
 0001:0000335C       @LStrFromString
 0001:00003380       @LStrFromWStr
 0001:00003198       @LStrLAsg
 0001:000033B8       @LStrLen
 0001:00003698       @LStrPos
 0001:000036E0       @LStrSetLength
 0001:000035B0       @LStrToPChar
 0001:00003394       @LStrToString
 0001:000031C4       @NewAnsiString
 0001:0000376C       @NewWideString
 0001:00001EA0       @Pow10
 0001:00002B00       @RaiseAgain
 0001:00002AD8       @RaiseExcept
 0001:00001708       @ReallocMem
 0001:000018F8       @RewritText
 0001:00001878       @ROUND
 0001:000030F4       @RunError
 0001:00001E84       @SetEq
 0001:00002DE4       @StartLib
 0001:000002BC       @strlen
 0001:00002B84       @TryFinallyExit
 0001:00003608       @UniqueStringA
 0001:00004138       @ValInt64
 0001:00001CA4       @ValLong
 0001:00003E78       @VarClear
 0001:00003F30       @VarClr
 0001:00003F24       @VarCmpEQ
 0001:00003E80       @VarCopy
 0001:00003EEC       @VarFromBool
 0001:00003EFC       @VarFromCurr
 0001:00003F1C       @VarFromDisp
 0001:00003ED0       @VarFromInt
 0001:00003ED8       @VarFromInt64
 0001:00003F14       @VarFromIntf
 0001:00003F04       @VarFromLStr
 0001:00003EF4       @VarFromReal
 0001:00003F0C       @VarFromWStr
 0001:00003E98       @VarToBool
 0001:00003EA8       @VarToCurr
 0001:00003EC8       @VarToDisp
 0001:00003E88       @VarToInt
 0001:00003E90       @VarToInt64
 0001:00003EC0       @VarToIntf
 0001:00003EB0       @VarToLStr
 0001:00003EA0       @VarToReal
 0001:00003EB8       @VarToWStr
 0001:00001DB4       @WriteBytes
 0001:00003744       @WriteLString
 0001:00001E08       @WriteSpaces
 0001:000037AC       @WStrArrayClr
 0001:000037D0       @WStrAsg
 0001:0000390C       @WStrCat
 0001:00003794       @WStrClr
 0001:0000396C       @WStrCmp
 0001:000039F0       @WStrCopy
 0001:000038E0       @WStrFromLStr
 0001:000037F4       @WStrFromPCharLen
 0001:000038A4       @WStrFromPWChar
 0001:00003880       @WStrFromPWCharLen
 0001:00003900       @WStrLen
 0001:00003A3C       @WStrSetLength
 0001:000038F0       @WStrToPWChar
 0001:000017DC       @_IOTest
 0001:00003F64       @_lldiv
 0001:0000402C       @_llmod
 0001:00003F40       @_llmul
 0001:000040F8       @_llshl
 0001:00003FE0       @_lludiv
 0001:000040A8       @_llumod
 0001:00004118       @_llushr
 0001:000081F0       AbstractErrorHandler
 0002:00001028       AbstractErrorProc
 0002:00000100       AccessMode
 0001:0000EDEC       ActiveX
 0001:000003E0       AddBlockAfter
 0001:00004B70       AddModuleUnloadProc
 0001:00004B80       AddModuleUnloadProc
 0001:0000652C       AllocMem
 0002:000015AC       AllocMemCount
 0002:000015B0       AllocMemSize
 0001:000052C0       AllocTlsBuffer
 0001:00015BFC       AncestorValid
 0001:00006620       AnsiCompareStr
 0001:00006658       AnsiCompareText
 0001:000087A0       AnsiPos
 0001:000087D8       AnsiStrPos
 0001:00008878       AnsiStrRScan
 0001:000088A0       AnsiStrScan
 0001:00005120       AnsiToUtf8
 0001:0000A530       AnyChangeType
 0001:0000B928       AnyOp
 0001:0000AF5C       AnyToIntf
 0001:000081D4       AssertErrorHandler
 0002:00001020       AssertErrorProc
 0001:0000E484       AssignLongStr
 0001:0000EB00       AssignVariant
 0002:00001600       avail
 0001:000069B0       BackfillGetDiskFreeSpaceEx
 0002:000003C8       BaseTypeMap
 0002:000015D8       blockDescBlockList
 0002:000015DC       blockDescFreeList
 0002:00000458       BooleanIdents
 0001:00008708       ByteType
 0001:00008690       ByteTypeTest
 0002:00000438       CBooleanToRelationship
 0002:0000186C       ChangeAnyProc
 0001:0000A598       ChangeSourceAny
 0001:00003220       CharFromWChar
 0001:00008764       CharLength
 0001:000055D4       CharNext
 0001:00000234       CharNext
 0001:00002768       CheckJmp
 0001:0000C570       CheckType
 0001:0000B9B4       CheckType
 0002:00000434       CInvalidCustomVariantType
 0001:000179D4       Classes
 0001:00010088       ClassNotFound
 0002:00001868       ClearAnyProc
 0001:0000D864       ClearVariantTypeList
 0001:000001D4       CloseHandle
 0001:00005494       CloseHandle
 0002:0000103C       CmdLine
 0002:00001038       CmdShow
 0001:00010338       CollectionsEqual
 0001:000006C0       Commit
 0002:0000161C       committedRoot
 0001:00006588       CompareMem
 0001:0000549C       CompareString
 0001:000065A8       CompareText
 0001:00013498       ComponentCreated
 0001:00007C44       ConvertAddr
 0001:00006508       ConvertErrorFmt
 0001:0000436C       CopyArray
 0001:00008118       CreateAssertException
 0001:000082A0       CreateAVObject
 0001:00013518       CreateComponent
 0001:000054A4       CreateEvent
 0001:000054AC       CreateFile
 0001:000001DC       CreateFileA
 0001:00008044       CreateInOutError
 0002:00000444       CRelationshipToBoolean
 0002:000000F8       cSimpleBoolStrs
 0002:00001614       curAlloc
 0002:00001738       CurrencyDecimals
 0002:00001734       CurrencyFormat
 0002:00001730       CurrencyString
 0002:000002C0       CVarTypeToElementInfo
 0002:00001739       DateSeparator
 0002:00000134       DCon10
 0002:00000014       DebugHook
 0002:00001737       DecimalSeparator
 0001:0000D188       DecIndices
 0001:00000754       Decommit
 0001:00000D70       DecommitFree
 0002:000015F0       decommittedRoot
 0002:0000000C       Default8087CW
 0002:00000020       DefaultTextLineBreakStyle
 0002:000001B4       DefLongDayNames
 0002:00000168       DefLongMonthNames
 0002:00000198       DefShortDayNames
 0002:00000138       DefShortMonthNames
 0001:000046C4       DelayLoadResourceModule
 0001:00000410       DeleteBlock
 0001:00000380       DeleteCriticalSection
 0001:000054B4       DeleteCriticalSection
 0001:00000BB8       DeleteFree
 0002:0000007C       dig
 0002:00001000       DispCallByIDProc
 0002:00001714       DllProc
 0001:000085CC       DoneExceptions
 0002:00000460       DotSep
 0001:0001115C       DoWrite
 0001:0000D134       DynArrayBounds
 0001:00004384       DynArrayClear
 0001:0000D0AC       DynArrayDim
 0001:0000D090       DynArrayElTypeInfo
 0001:0000D588       DynArrayFromVariant
 0001:0000D050       DynArrayIndex
 0001:0000438C       DynArraySetLength
 0001:0000D0C4       DynArraySize
 0001:0000D274       DynArrayToVariant
 0001:0000D1F4       DynArrayVariantBounds
 0001:0000D24C       DynArrayVarType
 0001:00008018       EHeapException.FreeInstance
 0002:00001854       EmptyParam
 0002:000000B4       EmptyStr
 0002:000000B8       EmptyWideStr
 0001:00017CFC       Eng
 0001:00000370       EnterCriticalSection
 0001:000054BC       EnterCriticalSection
 0001:000054C4       EnumCalendarInfoA
 0001:000078B8       EnumEraNames
 0001:000078F4       EnumEraYearOffsets
 0002:00001800       EraNames
 0002:0000181C       EraYearOffsets
 0002:00000074       errCaption
 0001:000017D0       Error
 0002:00000004       ErrorAddr
 0001:00001784       ErrorAt
 0001:000080C4       ErrorHandler
 0002:000001D0       ErrorMap
 0002:00001008       ErrorProc
 0002:000013E0       ErrOutput
 0002:0000100C       ExceptClsProc
 0001:00008538       ExceptHandler
 0001:00007E8C       Exception.Create
 0001:00007EC8       Exception.CreateFmt
 0001:00007F48       Exception.CreateRes
 0001:00007F84       Exception.CreateResFmt
 0002:0000101C       ExceptionClass
 0001:00007C50       ExceptionErrorMessage
 0002:00000208       ExceptMap
 0001:00001758       ExceptObject
 0002:00001010       ExceptObjProc
 0002:00001004       ExceptProc
 0002:00000000       ExitCode
 0001:00002F54       ExitDll
 0002:00001040       ExitProc
 0001:0000023C       ExitProcess
 0002:00001024       ExitProcessProc
 0001:0000536C       ExitProcessTLS
 0001:00005344       ExitThreadTLS
 0001:00006978       ExtractFileName
 0001:0000B924       Failure
 0002:0000183C       FalseBoolStrs
 0002:00000128       FCon1E18
 0001:00006920       FileClose
 0001:00006888       FileCreate
 0001:00006864       FileCreate
 0002:00000008       FileMode
 0001:00001940       FileNOPProc
 0001:00006808       FileOpen
 0001:00006890       FileRead
 0002:00000464       FilerSignature
 0001:000068E8       FileSeek
 0001:000068BC       FileWrite
 0001:00000CA0       FillAfterGap
 0001:00000C4C       FillBeforeGap
 0001:00000D38       FillerSizeAfterGap
 0001:00000CC8       FillerSizeBeforeGap
 0001:00009A0C       Finalization
 0001:00009C6C       Finalization
 0001:00005424       Finalization
 0001:0000545C       Finalization
 0001:00017F48       Finalization
 0001:0000DFB8       Finalization
 0001:0000DCA0       Finalization
 0001:00005934       Finalization
 0001:0000566C       Finalization
 0001:0001792C       Finalization
 0001:00005634       Finalization
 0001:0000ED64       Finalization
 0001:0000EDBC       Finalization
 0001:000051C8       Finalization
 0001:0000437C       FinalizeArray
 0001:00002D24       FinalizeUnits
 0001:0001536C       FindAncestor
 0001:00004734       FindBS
 0001:0000024C       FindClose
 0001:00000C1C       FindCommitted
 0001:0000DBA4       FindCustomVariantType
 0001:0000DB04       FindCustomVariantType
 0001:000136C8       FindExistingComponent
 0001:00000254       FindFirstFile
 0001:0001028C       FindGlobalComponent
 0002:000019F4       FindGlobalComponentProcs
 0001:0000469C       FindHInstance
 0001:00010210       FindIdentToInt
 0001:00010194       FindIntToIdent
 0001:00012BEC       FindNestedComponent
 0001:0000470C       FindResourceHInstance
 0002:0000184C       FLanguages
 0001:0000746C       FloatToDecimal
 0001:00007194       FloatToText
 0001:00001BA4       Flush
 0001:00007090       FmtStr
 0001:0000707C       Format
 0001:00006C28       FormatBuf
 0001:00006C1C       FormatClearStr
 0001:00006BB0       FormatError
 0002:00000120       FormatErrorStrs
 0001:000054CC       FormatMessage
 0001:00006C08       FormatVarToStr
 0001:00001E98       FPower10
 0001:00009670       FreeAndNil
 0001:00000988       FreeCommitted
 0001:00000EA8       FreeCurAlloc
 0001:000178B8       FreeIntConstList
 0001:0000025C       FreeLibrary
 0001:00000608       FreeSpace
 0001:00008F6C       FreeTerminateProcs
 0001:000054D4       GetACP
 0001:00000388       GetBlockDesc
 0001:000100F4       GetClass
 0001:00000324       GetCmdShow
 0001:00000264       GetCommandLine
 0001:000007D4       GetCommitted
 0001:00000864       GetCommittedAt
 0001:000161B4       GetComponentValue
 0001:000054DC       GetCPInfo
 0001:0000031C       GetCurrentThreadId
 0001:000054E4       GetCurrentThreadId
 0001:00010AAC       GetDesigner
 0001:000054EC       GetDiskFreeSpaceA
 0002:000000F4       GetDiskFreeSpaceEx
 0001:000024F0       GetDynaMethod
 0001:0000E028       GetEnumName
 0001:0000E11C       GetEnumNameValue
 0001:0000E168       GetEnumValue
 0001:0000796C       GetEraNamesAndYearOffsets
 0001:00008288       GetExceptionClass
 0001:0000846C       GetExceptionObject
 0001:0001007C       GetFieldClassTable
 0001:000001EC       GetFileSize
 0001:000001E4       GetFileType
 0001:0000E7F0       GetFloatProp
 0001:00008B40       GetFormatSettings
 0001:0000EC0C       GetInt64Prop
 0001:0000EC70       GetInterfaceProp
 0001:00002180       GetKeyboardType
 0001:000054F4       GetLastError
 0001:0000026C       GetLastError
 0001:00007730       GetLocaleChar
 0001:00000274       GetLocaleInfo
 0001:000054FC       GetLocaleInfo
 0001:000076E4       GetLocaleStr
 0001:0000E498       GetLongStrProp
 0001:0000EB94       GetMethodProp
 0001:00005504       GetModuleFileName
 0001:0000027C       GetModuleFileName
 0001:00000284       GetModuleHandle
 0001:0000550C       GetModuleHandle
 0001:00007794       GetMonthDayNames
 0001:0000E2C0       GetOrdProp
 0001:0000028C       GetProcAddress
 0001:00005514       GetProcAddress
 0001:0000E1CC       GetPropInfo
 0001:0000E23C       GetPropInfos
 0001:0000E390       GetShortStrProp
 0001:0000E428       GetShortStrPropAsLongStr
 0001:0000052C       GetSpace
 0001:00000590       GetSpaceAt
 0001:00000294       GetStartupInfo
 0001:000001F4       GetStdHandle
 0001:0000551C       GetStdHandle
 0001:00005524       GetStringTypeEx
 0001:0000E5C8       GetStrProp
 0001:00017BA4       GetSysDir
 0001:0000552C       GetSystemDirectory
 0001:000055DC       GetSystemMetrics
 0001:0000029C       GetThreadLocale
 0001:00005534       GetThreadLocale
 0001:0000553C       GetTickCount
 0001:000052CC       GetTlsSize
 0001:0000E01C       GetTypeData
 0001:0000CCBC       GetVarArray
 0001:0000CB70       GetVarDataArrayInfo
 0001:00003E50       GetVariantManager
 0001:0000EB14       GetVariantProp
 0001:00005544       GetVersionEx
 0001:0000E634       GetWideStrProp
 0001:0000E518       GetWideStrPropAsLongStr
 0001:00017B2C       GetWinDir
 0001:0000554C       GetWindowsDirectory
 0001:00005554       GlobalAlloc
 0001:000055F4       GlobalAllocPtr
 0002:000019F8       GlobalFixupList
 0001:0000555C       GlobalFree
 0001:00005620       GlobalFreePtr
 0001:0000556C       GlobalHandle
 0001:00005564       GlobalLock
 0002:000019E4       GlobalNameSpace
 0001:00005574       GlobalReAlloc
 0001:00005604       GlobalReAllocPtr
 0001:0000557C       GlobalUnlock
 0002:00001924       GOldVariantManager
 0002:00001878       GVariantManager
 0001:00013D90       HandleException
 0002:00000010       HeapAllocFlags
 0002:000015BC       heapErrorCode
 0002:000015C0       heapLock
 0002:000000F0       HexDisplayPrefix
 0002:00001710       HInstance
 0001:00009EC4       Increment
 0001:00000A14       InitAllocator
 0002:0000162C       InitContext
 0001:00008F8C       InitDriveSpacePtr
 0001:00008548       InitExceptions
 0001:00005584       InitializeCriticalSection
 0001:00000368       InitializeCriticalSection
 0002:000015B8       initialized
 0001:000053D0       InitializeModule
 0001:00008954       InitLeadBytes
 0001:00008638       InitPlatformId
 0001:00005318       InitProcessTLS
 0001:000089CC       InitSysLocale
 0001:000052D4       InitThreadTLS
 0001:00002D84       InitUnits
 0001:00003E30       InitVariantManager
 0002:00001048       Input
 0001:00000E20       InsertFree
 0001:0000C5A8       Int64Compare
 0001:0000BBB0       Int64Op
 0001:0000C594       IntCompare
 0002:000019EC       IntConstList
 0001:00000314       InterlockedDecrement
 0001:00008FF4       InterlockedDecrement
 0001:00009000       InterlockedExchange
 0001:00009008       InterlockedExchangeAdd
 0001:0000030C       InterlockedIncrement
 0001:00008FE8       InterlockedIncrement
 0001:00001980       InternalClose
 0001:00001B5C       InternalFlush
 0001:00000C7C       InternalFreeMem
 0001:000035BC       InternalUniqueString
 0001:0000BA8C       IntOp
 0001:00006724       IntToStr
 0001:000066F4       IntToStr
 0002:00001848       InvalidPointer
 0001:000023C4       InvokeImplGetter
 0001:0000180C       IOResult
 0002:00001044       IsConsole
 0001:000160A8       IsDefault
 0001:00016324       IsDefault
 0001:000165B4       IsDefaultValue
 0001:000167A8       IsDefaultValue
 0001:00015E3C       IsDefaultValue
 0001:000168E0       IsDefaultValue
 0001:00016010       IsDefaultValue
 0001:00015F6C       IsDefaultValue
 0001:0000D0CC       IsDynArrayRectangular
 0002:00001034       IsLibrary
 0002:00001045       IsMultiThread
 0001:0000E290       IsStoredProp
 0001:00006690       IsValidIdent
 0001:000089B4       IsWesternGroup
 0002:00000018       JITEnable
 0001:00006928       LastDelimiter
 0001:000088E0       LCIDToCodePage
 0002:000000D0       LeadBytes
 0001:0000558C       LeaveCriticalSection
 0001:00000378       LeaveCriticalSection
 0002:00000024       LibModuleList
 0002:000017FE       ListSeparator
 0001:000002A4       LoadLibraryEx
 0001:00004900       LoadResourceModule
 0001:00005170       LoadResString
 0001:000055E4       LoadString
 0001:000002AC       LoadString
 0001:00005290       LocalAlloc
 0001:00000348       LocalAlloc
 0001:00005298       LocalFree
 0001:00000350       LocalFree
 0001:00007758       LocalGetLocaleStr
 0002:00001740       LongDateFormat
 0002:000017D4       LongDayNames
 0002:00001788       LongMonthNames
 0002:00001754       LongTimeFormat
 0001:0000654C       LowerCase
 0001:000002B4       lstrcpyn
 0002:000019D0       LVarTypes
 0002:000019D4       LVarTypeSync
 0002:0000102C       MainInstance
 0002:00001030       MainThreadID
 0001:000003D8       MakeEmpty
 0001:00002EF8       MakeErrorMessage
 0001:00008208       MapException
 0001:00002B9C       MapToRunError
 0002:0000002C       MemoryManager
 0001:00000428       MergeBlockAfter
 0001:00000EF4       MergeCommit
 0001:000055EC       MessageBox
 0001:00000244       MessageBox
 0001:0000569C       Messages
 0002:0000008C       Module
 0002:00001705       ModuleIsCpp
 0002:00001704       ModuleIsLib
 0001:00017924       ModuleUnload
 0002:00000028       ModuleUnloadList
 0001:0000182C       Move
 0001:00017A38       MsgBox
 0001:000002C4       MultiByteToWideChar
 0002:00001735       NegCurrFormat
 0001:00000F80       NewCommit
 0001:00000FAC       NewCommitAt
 0002:00000468       NilMethod
 0002:0000001C       NoErrMsg
 0001:00002754       NotifyAnyExcept
 0001:00010B44       NotifyDesigner
 0001:00002728       NotifyExcept
 0001:00002788       NotifyExceptFinally
 0001:00004C00       NotifyModuleUnload
 0001:00002704       NotifyNonDelphiException
 0001:00002740       NotifyOnExcept
 0001:000026E8       NotifyReRaise
 0001:000027B0       NotifyTerminate
 0001:000027CC       NotifyUnhandled
 0001:0000DC8C       Null
 0001:000162DC       ObjectAncestorMatch
 0001:00003DC8       OleStrToStrVar
 0001:0000B410       OleVarFromAny
 0001:0000B474       OleVarFromVarArrayProc
 0001:000018A0       OpenText
 0002:000003E0       OpTypeMap
 0002:00001844       OutOfMemory
 0002:00001214       Output
 0001:0001619C       OwnedBy
 0001:00017FE8       pluginexample
 0001:0000FDD4       PointerInModule
 0001:00012E08       PropertyNotFound
 0001:00013E90       PropPathError
 0001:00012DFC       PropValueError
 0001:00007150       PutExponent
 0001:000081C4       RaiseAssertException
 0001:000123BC       RaiseException
 0001:000001FC       RaiseException
 0002:00001014       RaiseExceptionProc
 0001:00008EC0       RaiseLastOSError
 0001:00014CE0       ReadCustomVariant
 0001:00012DE4       ReadError
 0001:00005594       ReadFile
 0001:00000204       ReadFile
 0001:0000C5E4       RealCompare
 0001:0000B9FC       RealOp
 0001:000134B8       Recover
 0002:00001870       RefAnyProc
 0001:000002CC       RegCloseKey
 0002:000019F0       RegGroups
 0001:00004C5C       RegisterModule
 0001:000002D4       RegOpenKeyEx
 0001:000002DC       RegQueryValueEx
 0002:00000038       reMap
 0002:00001610       remBytes
 0001:0000049C       RemoveBlock
 0001:00012CB4       RemoveFixupReferences
 0001:00012D60       RemoveFixups
 0001:00013040       RemoveGlobalFixup
 0001:00004BA0       RemoveModuleUnloadProc
 0001:00004B78       RemoveModuleUnloadProc
 0001:0000559C       ResetEvent
 0001:00001434       ResizeInPlace
 0001:00010528       ReturnAddr
 0001:000112BC       ReturnAddr
 0002:0000160C       rover
 0001:0000DFE8       RTLConsts
 0001:0000020C       RtlUnwind
 0002:00001018       RTLUnwindProc
 0002:00000054       runErrMsg
 0001:00001778       RunErrorAt
 0001:00009C34       SafeArrayCreate
 0001:00009C54       SafeArrayGetElement
 0001:00009C44       SafeArrayGetLBound
 0001:00009C4C       SafeArrayGetUBound
 0001:00009C64       SafeArrayPtrOfIndex
 0001:00009C5C       SafeArrayPutElement
 0001:00009C3C       SafeArrayRedim
 0001:000065FC       SameText
 0001:00000FE0       SearchSmallBlocks
 0001:0000CAE0       SetClearVarToEmptyParam
 0001:00013628       SetCompName
 0001:000055A4       SetEndOfFile
 0001:00000214       SetEndOfFile
 0001:000055AC       SetEvent
 0001:00002CDC       SetExceptionHandler
 0001:0000021C       SetFilePointer
 0001:000055B4       SetFilePointer
 0001:0000E908       SetFloatProp
 0001:000017FC       SetInOutRes
 0001:0000EC34       SetInt64Prop
 0001:0000ECF0       SetInterfaceProp
 0001:00014114       SetInterfaceReference
 0001:0001408C       SetIntIdent
 0001:0000E4D8       SetLongStrProp
 0001:0000EBD4       SetMethodProp
 0001:000140D4       SetObjectIdent
 0001:0000E334       SetOrdProp
 0001:0000E3D4       SetShortStrProp
 0001:0000E450       SetShortStrPropAsLongStr
 0001:0000E608       SetStrProp
 0001:00003E64       SetVariantManager
 0001:0000EB54       SetVariantProp
 0001:0000E71C       SetWideStrProp
 0001:0000E570       SetWideStrPropAsLongStr
 0002:0000010C       ShareMode
 0002:0000173C       ShortDateFormat
 0002:000017B8       ShortDayNames
 0002:00001758       ShortMonthNames
 0002:00001750       ShortTimeFormat
 0001:00007DD8       ShowException
 0001:0000C684       SimpleVarCmp
 0001:00014814       SkipBinary
 0001:00014844       SkipCollection
 0001:000147EC       SkipList
 0001:00008EB8       Sleep
 0002:00001618       smallTab
 0002:000015E0       spaceRoot
 0001:00006B70       StrAlloc
 0001:0000872C       StrByteType
 0001:00008744       StrCharLength
 0001:00006A80       StrComp
 0001:0000C60C       StringCompare
 0001:00012258       StringListCompareStrings
 0001:00003DEC       StringToOleStr
 0001:00006A4C       StrLCopy
 0001:00006A24       StrLen
 0001:0000703C       StrLFmt
 0001:00006AA4       StrLIComp
 0001:00006A3C       StrMove
 0001:00006B84       StrNew
 0001:00006B5C       StrPas
 0001:00006B08       StrPos
 0001:00006AE8       StrScan
 0001:00006758       StrToInt
 0001:000067AC       StrToInt64
 0001:00006794       StrToIntDef
 0001:00017C34       StrToStrList
 0001:000096A4       Supports
 0001:00009680       Supports
 0002:0000049C       SyncList
 0001:000002F4       SysAllocStringLen
 0001:00005964       SysConst
 0001:00007698       SysErrorMessage
 0001:00001290       SysFreeMem
 0001:00000304       SysFreeString
 0001:00001100       SysGetMem
 0001:00005454       SysInit
 0002:000017F0       SysLocale
 0001:00001604       SysReallocMem
 0001:000002FC       SysReAllocStringLen
 0001:0000521C       System
 0001:00009B8C       SysUtils
 0001:0000FFF4       TClassFinder.GetClass
 0001:00010BF4       TCollection.Add
 0001:00010F58       TCollection.Added
 0001:00010C00       TCollection.Assign
 0001:00010C98       TCollection.BeginUpdate
 0001:00010C9C       TCollection.Changed
 0001:00010CAC       TCollection.Clear
 0001:00010F5C       TCollection.Deleting
 0001:00010BA8       TCollection.Destroy
 0001:00010D14       TCollection.EndUpdate
 0001:00010D24       TCollection.GetAttr
 0001:00010D20       TCollection.GetAttrCount
 0001:00010D50       TCollection.GetCount
 0001:00010D58       TCollection.GetItem
 0001:00010D30       TCollection.GetItemAttr
 0001:00010D6C       TCollection.GetNamePath
 0001:00010E34       TCollection.GetPropName
 0001:00010F60       TCollection.Notify
 0001:00010F50       TCollection.SetItemName
 0001:00010F54       TCollection.Update
 0001:00017210       TComponent.BeforeDestruction
 0001:000176DC       TComponent.ChangeName
 0001:0001714C       TComponent.Create
 0001:00017470       TComponent.DefineProperties
 0001:00017198       TComponent.Destroy
 0001:00017340       TComponent.DestroyComponents
 0001:00017398       TComponent.Destroying
 0001:000177C4       TComponent.ExecuteAction
 0001:00017600       TComponent.FindComponent
 0001:00017504       TComponent.GetChildOwner
 0001:00017508       TComponent.GetChildParent
 0001:000174FC       TComponent.GetChildren
 0001:000176F0       TComponent.GetComponent
 0001:0001771C       TComponent.GetComponentCount
 0001:0001750C       TComponent.GetNamePath
 0001:00017520       TComponent.GetOwner
 0001:00017528       TComponent.GetParentComponent
 0001:000174F8       TComponent.HasParent
 0001:0001725C       TComponent.Insert
 0001:000172B0       TComponent.InsertComponent
 0001:000178B4       TComponent.IntfGetComponent
 0001:00017548       TComponent.Loaded
 0001:00017414       TComponent.Notification
 0001:00017554       TComponent.PaletteCreated
 0001:00017834       TComponent.QueryInterface
 0001:0001721C       TComponent.ReadLeft
 0001:00017558       TComponent.ReadState
 0001:00017230       TComponent.ReadTop
 0001:00017288       TComponent.Remove
 0001:00017308       TComponent.RemoveComponent
 0001:000173F8       TComponent.RemoveFreeNotification
 0001:000173D4       TComponent.RemoveNotification
 0001:00017814       TComponent.SafeCallException
 0001:00017524       TComponent.SetChildOrder
 0001:0001772C       TComponent.SetDesigning
 0001:00017650       TComponent.SetName
 0001:0001752C       TComponent.SetParentComponent
 0001:0001777C       TComponent.SetReference
 0001:000177EC       TComponent.UpdateAction
 0001:0001753C       TComponent.Updated
 0001:0001782C       TComponent.UpdateRegistry
 0001:00017530       TComponent.Updating
 0001:000175E8       TComponent.ValidateContainer
 0001:000175FC       TComponent.ValidateInsert
 0001:00017568       TComponent.ValidateRename
 0001:00017244       TComponent.WriteLeft
 0001:00017560       TComponent.WriteState
 0001:00017250       TComponent.WriteTop
 0001:00017874       TComponent._AddRef
 0001:00017894       TComponent._Release
 0001:0001279C       TCustomMemoryStream.Read
 0001:000127D4       TCustomMemoryStream.Seek
 0001:00012794       TCustomMemoryStream.SetPointer
 0001:0000D8D4       TCustomVariantType.BinaryOp
 0001:0000D8E0       TCustomVariantType.Cast
 0001:0000D918       TCustomVariantType.CastTo
 0001:0000D9A4       TCustomVariantType.CastToOle
 0001:0000D960       TCustomVariantType.Compare
 0001:0000D96C       TCustomVariantType.CompareOp
 0001:0000D9E0       TCustomVariantType.Destroy
 0001:0000DAB8       TCustomVariantType.DispInvoke
 0001:0000DA64       TCustomVariantType.IsClear
 0001:0000DA68       TCustomVariantType.LeftPromotion
 0001:0000DA7C       TCustomVariantType.OlePromotion
 0001:0000DADC       TCustomVariantType.QueryInterface
 0001:0000DA84       TCustomVariantType.RaiseCastError
 0001:0000DA94       TCustomVariantType.RaiseDispError
 0001:0000DA8C       TCustomVariantType.RaiseInvalidOp
 0001:0000DA9C       TCustomVariantType.RightPromotion
 0001:0000DAB0       TCustomVariantType.UnaryOp
 0001:0000DAC4       TCustomVariantType._AddRef
 0001:0000DAD0       TCustomVariantType._Release
 0002:000002BC       TerminateProcList
 0002:00001046       Test8086
 0001:00001990       TextClose
 0001:00001904       TextIn
 0001:000019B0       TextOpen
 0001:00001944       TextOut
 0001:0001296C       TFiler.Create
 0001:000129B4       TFiler.Destroy
 0001:000129DC       TFiler.SetRoot
 0001:00012698       TFileStream.Create
 0001:00012654       TFileStream.Create
 0001:00012760       TFileStream.Destroy
 0001:00012590       THandleStream.Create
 0001:000125CC       THandleStream.Read
 0001:000125EC       THandleStream.Seek
 0001:00012618       THandleStream.SetSize
 0001:0001262C       THandleStream.SetSize
 0001:000125DC       THandleStream.Write
 0002:00001736       ThousandSeparator
 0002:000019FC       ThreadLock
 0002:00001748       TimeAMString
 0002:0000174C       TimePMString
 0002:00001744       TimeSeparator
 0001:00004D20       TInterfacedObject.AfterConstruction
 0001:00004D2C       TInterfacedObject.BeforeDestruction
 0001:00004D3C       TInterfacedObject.NewInstance
 0001:00004D4C       TInterfacedObject.QueryInterface
 0001:00004D74       TInterfacedObject._AddRef
 0001:00004D88       TInterfacedObject._Release
 0001:0001047C       TList.Add
 0001:000104B0       TList.Clear
 0001:000104C8       TList.Delete
 0001:0001045C       TList.Destroy
 0001:0001052C       TList.Error
 0001:00010564       TList.Error
 0001:000105B8       TList.Get
 0001:000105E0       TList.Grow
 0001:00010614       TList.IndexOf
 0001:00010634       TList.Last
 0001:00010760       TList.Notify
 0001:00010640       TList.Put
 0001:00010694       TList.Remove
 0001:000106B4       TList.SetCapacity
 0001:000106F0       TList.SetCount
 0001:000052A0       TlsAlloc
 0002:0000171C       tlsBuffer
 0001:000052A8       TlsFree
 0001:000052B0       TlsGetValue
 0002:00001708       TlsIndex
 0002:FFBE700C       TlsLast
 0002:000000A4       TlsProc
 0001:000052B8       TlsSetValue
 0001:00012824       TMemoryStream.Clear
 0001:000127F8       TMemoryStream.Destroy
 0001:00012890       TMemoryStream.Realloc
 0001:0001283C       TMemoryStream.SetCapacity
 0001:00012864       TMemoryStream.SetSize
 0001:0001291C       TMemoryStream.Write
 0001:0000953C       TMultiReadExclusiveWriteSynchronizer.BeginRead
 0001:00009398       TMultiReadExclusiveWriteSynchronizer.BeginWrite
 0001:00009354       TMultiReadExclusiveWriteSynchronizer.BlockReaders
 0001:00009298       TMultiReadExclusiveWriteSynchronizer.Create
 0001:0000930C       TMultiReadExclusiveWriteSynchronizer.Destroy
 0001:000095E0       TMultiReadExclusiveWriteSynchronizer.EndRead
 0001:00009498       TMultiReadExclusiveWriteSynchronizer.EndWrite
 0001:0000936C       TMultiReadExclusiveWriteSynchronizer.UnblockOneWriter
 0001:00009360       TMultiReadExclusiveWriteSynchronizer.UnblockReaders
 0001:00009378       TMultiReadExclusiveWriteSynchronizer.WaitForReadSignal
 0001:00009388       TMultiReadExclusiveWriteSynchronizer.WaitForWriteSignal
 0001:00002560       TObject.AfterConstruction
 0001:00002564       TObject.BeforeDestruction
 0001:0000254C       TObject.ClassInfo
 0001:00002290       TObject.ClassName
 0001:000022A4       TObject.ClassNameIs
 0001:000022CC       TObject.ClassParent
 0001:00002288       TObject.ClassType
 0001:000023A4       TObject.CleanupInstance
 0001:00002310       TObject.Create
 0001:0000255C       TObject.DefaultHandler
 0001:00002330       TObject.Destroy
 0001:00002568       TObject.Dispatch
 0001:00002620       TObject.FieldAddress
 0001:00002340       TObject.Free
 0001:000022F4       TObject.FreeInstance
 0001:000023F4       TObject.GetInterface
 0001:00002488       TObject.GetInterfaceEntry
 0001:00002538       TObject.InheritsFrom
 0001:0000234C       TObject.InitInstance
 0001:00002308       TObject.InstanceSize
 0001:00002590       TObject.MethodAddress
 0001:000025E0       TObject.MethodName
 0001:000022D8       TObject.NewInstance
 0001:00002554       TObject.SafeCallException
 0001:00004748       ToLongPath
 0001:00010908       TPersistent.Assign
 0001:0001091C       TPersistent.AssignError
 0001:000109EC       TPersistent.AssignTo
 0001:000109F4       TPersistent.DefineProperties
 0001:000108DC       TPersistent.Destroy
 0001:000109F8       TPersistent.GetNamePath
 0001:00010AA8       TPersistent.GetOwner
 0001:00012AB8       TPropFixup.Create
 0001:00012B10       TPropFixup.MakeGlobalReference
 0001:00012B58       TPropFixup.ResolveReference
 0001:00012B68       TPropIntfFixup.ResolveReference
 0001:00007A1C       TranslateDateFormat
 0001:00012E70       TReader.CheckValue
 0001:00012EC8       TReader.DefineBinaryProperty
 0001:00012E94       TReader.DefineProperty
 0001:00012E34       TReader.Destroy
 0001:000130BC       TReader.DoFixupReferences
 0001:00012FA4       TReader.EndOfList
 0001:00012FB8       TReader.Error
 0001:00014B2C       TReader.FindAncestorComponent
 0001:00014C24       TReader.FindComponentClass
 0001:00012FD8       TReader.FindMethod
 0001:000131DC       TReader.FlushBuffer
 0001:00013200       TReader.FreeFixups
 0001:0001323C       TReader.GetFieldClass
 0001:000132D0       TReader.GetPosition
 0001:000132E8       TReader.NextValue
 0001:000132F8       TReader.PropertyError
 0001:0001330C       TReader.Read
 0001:00013358       TReader.ReadBuffer
 0001:00013394       TReader.ReadChar
 0001:000133EC       TReader.ReadCollection
 0001:0001376C       TReader.ReadComponent
 0001:00013B04       TReader.ReadCurrency
 0001:00013944       TReader.ReadData
 0001:000139B4       TReader.ReadDataInner
 0001:00013B50       TReader.ReadDate
 0001:00013A84       TReader.ReadFloat
 0001:00013B90       TReader.ReadIdent
 0001:00013CFC       TReader.ReadInt64
 0001:00013C90       TReader.ReadInteger
 0001:00013D40       TReader.ReadListBegin
 0001:00013D48       TReader.ReadListEnd
 0001:00013D50       TReader.ReadPrefix
 0001:00013EAC       TReader.ReadProperty
 0001:000141D4       TReader.ReadPropValue
 0001:000144F8       TReader.ReadSet
 0001:00013AC4       TReader.ReadSingle
 0001:000145B4       TReader.ReadStr
 0001:000145F0       TReader.ReadString
 0001:00014790       TReader.ReadValue
 0001:00014EA0       TReader.ReadVariant
 0001:000146AC       TReader.ReadWideString
 0001:00014BE4       TReader.ReferenceName
 0001:00014BFC       TReader.SetName
 0001:00014C98       TReader.SkipBytes
 0001:00014A84       TReader.SkipComponent
 0001:00014A3C       TReader.SkipProperty
 0001:000147A4       TReader.SkipSetBody
 0001:000148A0       TReader.SkipValue
 0001:0000FCB8       TRegGroup.Create
 0001:0000FD34       TRegGroup.Destroy
 0001:0000FD74       TRegGroup.GetClass
 0001:0000FDF4       TRegGroup.UnregisterModuleClasses
 0001:0000FE98       TRegGroups.Create
 0001:0000FF0C       TRegGroups.Destroy
 0001:0000FF68       TRegGroups.GetClass
 0001:0000FFAC       TRegGroups.Lock
 0001:0000FFB8       TRegGroups.Unlock
 0001:0000FFC4       TRegGroups.UnregisterModuleClasses
 0002:00001838       TrueBoolStrs
 0001:0000100C       TryHarder
 0001:00001D70       TryOpenForOutput
 0001:000122D0       TStream.GetPosition
 0001:00012304       TStream.GetSize
 0001:0001248C       TStream.Seek
 0001:00012408       TStream.Seek
 0001:000122F0       TStream.SetPosition
 0001:00012368       TStream.SetSize
 0001:00012350       TStream.SetSize
 0001:00012354       TStream.SetSize64
 0001:000124FC       TStream.WriteBuffer
 0001:00012534       TStream.WriteDescendent
 0001:00011CF8       TStringList.Add
 0001:00011D04       TStringList.AddObject
 0001:00011D68       TStringList.Changed
 0001:00011D84       TStringList.Changing
 0001:00011DA0       TStringList.Clear
 0001:000122B4       TStringList.CompareStrings
 0001:0001227C       TStringList.CustomSort
 0001:00011DE0       TStringList.Delete
 0001:00011C9C       TStringList.Destroy
 0001:00011E4C       TStringList.Exchange
 0001:00011EA8       TStringList.ExchangeItems
 0001:00011ECC       TStringList.Find
 0001:00011F44       TStringList.Get
 0001:00011F78       TStringList.GetCapacity
 0001:00011F7C       TStringList.GetCount
 0001:00011F80       TStringList.GetObject
 0001:00011FA8       TStringList.Grow
 0001:00011FDC       TStringList.IndexOf
 0001:00012018       TStringList.Insert
 0001:0001207C       TStringList.InsertItem
 0001:00012028       TStringList.InsertObject
 0001:000120F4       TStringList.Put
 0001:00012150       TStringList.PutObject
 0001:00012190       TStringList.QuickSort
 0001:00012224       TStringList.SetCapacity
 0001:00012240       TStringList.SetUpdateState
 0001:0001226C       TStringList.Sort
 0001:00010FB4       TStrings.Add
 0001:00010FD8       TStrings.AddObject
 0001:00010FFC       TStrings.AddStrings
 0001:000110B4       TStrings.Assign
 0001:00011144       TStrings.BeginUpdate
 0001:00011C90       TStrings.CompareStrings
 0001:000111B4       TStrings.DefineProperties
 0001:00010F84       TStrings.Destroy
 0001:00011200       TStrings.EndUpdate
 0001:00011214       TStrings.Equals
 0001:000112F8       TStrings.Error
 0001:000112C0       TStrings.Error
 0001:00011350       TStrings.Exchange
 0001:00011438       TStrings.GetCapacity
 0001:00011440       TStrings.GetObject
 0001:00011444       TStrings.GetText
 0001:00011498       TStrings.GetTextStr
 0001:000115C0       TStrings.IndexOf
 0001:0001164C       TStrings.IndexOfName
 0001:00011714       TStrings.IndexOfObject
 0001:00011748       TStrings.InsertObject
 0001:00011778       TStrings.LoadFromFile
 0001:000117CC       TStrings.LoadFromStream
 0001:00011878       TStrings.Move
 0001:00011928       TStrings.Put
 0001:00011958       TStrings.PutObject
 0001:0001195C       TStrings.ReadData
 0001:00011A0C       TStrings.SaveToFile
 0001:00011A64       TStrings.SaveToStream
 0001:00011AC0       TStrings.SetCapacity
 0001:00011AC4       TStrings.SetStringsAdapter
 0001:00011AF8       TStrings.SetText
 0001:00011B48       TStrings.SetTextStr
 0001:00011C08       TStrings.SetUpdateState
 0001:00011C0C       TStrings.WriteData
 0001:00010834       TThreadList.Add
 0001:00010764       TThreadList.Create
 0001:000107B8       TThreadList.Destroy
 0001:000108BC       TThreadList.LockList
 0001:000108D0       TThreadList.UnlockList
 0001:00009144       TThreadLocalCounter.Close
 0001:00009010       TThreadLocalCounter.Create
 0001:000091CC       TThreadLocalCounter.Delete
 0001:0000904C       TThreadLocalCounter.Destroy
 0001:000090B4       TThreadLocalCounter.HashIndex
 0001:000090CC       TThreadLocalCounter.Open
 0001:00009214       TThreadLocalCounter.Reattach
 0001:00009240       TThreadLocalCounter.Recycle
 0001:000150C4       TWriter.AddAncestor
 0001:000150F8       TWriter.DefineBinaryProperty
 0001:000150D0       TWriter.DefineProperty
 0001:00015098       TWriter.Destroy
 0001:00015134       TWriter.FlushBuffer
 0001:00015124       TWriter.GetPosition
 0001:0001513C       TWriter.SetPosition
 0001:00015178       TWriter.SetRoot
 0001:00015190       TWriter.Write
 0001:000151DC       TWriter.WriteBinary
 0001:00015264       TWriter.WriteBuffer
 0001:0001527C       TWriter.WriteChar
 0001:000152CC       TWriter.WriteCollection
 0001:000153BC       TWriter.WriteComponent
 0001:00015908       TWriter.WriteCurrency
 0001:00015498       TWriter.WriteData
 0001:0001592C       TWriter.WriteDate
 0001:00015898       TWriter.WriteDescendent
 0001:000158C0       TWriter.WriteFloat
 0001:00015950       TWriter.WriteIdent
 0001:00015A14       TWriter.WriteInteger
 0001:00015A88       TWriter.WriteInteger
 0001:00015AE0       TWriter.WriteListBegin
 0001:00015AE8       TWriter.WriteListEnd
 0001:00016F98       TWriter.WriteMinStr
 0001:00015AF0       TWriter.WritePrefix
 0001:00015B34       TWriter.WriteProperties
 0001:000169DC       TWriter.WriteProperty
 0001:00016EEC       TWriter.WritePropName
 0001:00016F40       TWriter.WriteSignature
 0001:000158E4       TWriter.WriteSingle
 0001:00016F50       TWriter.WriteStr
 0001:00017030       TWriter.WriteString
 0001:00017138       TWriter.WriteValue
 0001:00016AF4       TWriter.WriteVariant
 0001:00017084       TWriter.WriteWideString
 0001:0000548C       Types
 0001:0000EDB4       TypInfo
 0001:00000224       UnhandledExceptionFilter
 0001:00004DB0       UnicodeToUtf8
 0001:00000AD8       UninitAllocator
 0001:00003600       UniqueString
 0001:00004C6C       UnregisterModule
 0001:00010148       UnRegisterModuleClasses
 0001:00002CFC       UnsetExceptionHandler
 0001:0000186C       UpCase
 0001:0000507C       UTF8Decode
 0001:00004FD0       UTF8Encode
 0001:00004E8C       Utf8ToUnicode
 0002:00000470       ValTypeToVarType
 0001:00009F20       VarArrayCopyForEach
 0001:0000A0E0       VarArrayCopyProc
 0001:0000CBBC       VarArrayCreate
 0001:0000CCE4       VarArrayDimCount
 0001:0000CEBC       VarArrayGet
 0001:0000CD34       VarArrayHighBound
 0001:0000CD0C       VarArrayLowBound
 0001:0000D028       VarArrayPut
 0001:00009DC8       VarCastError
 0001:0000A5B0       VarChangeType
 0001:0000C1B4       VarCompare
 0001:0000A0F4       VarCopyCommon
 0001:0000A214       VarCopyNoInd
 0002:00001864       VarDispProc
 0001:00009C2C       VariantChangeTypeEx
 0001:00009C14       VariantClear
 0001:00009C1C       VariantCopy
 0001:00009C24       VariantCopyInd
 0001:00009C0C       VariantInit
 0002:00001658       VariantManager
 0001:0000DD04       Variants
 0001:00003E18       VariantSystemDefaultVarClear
 0001:00003E10       VariantSystemUndefinedError
 0001:0000A21C       VarInt64FromVar
 0001:0000A3B8       VarInt64ToVar
 0001:00009DD0       VarInvalidOp
 0001:0000CD64       VarIsArray
 0001:0000CD5C       VarIsArray
 0001:0000CA0C       VarIsClear
 0001:0000CA9C       VarSameValue
 0001:0000B5F8       VarStrCat
 0001:0000A788       VarStringToOleStr
 0001:0000CA08       VarType
 0001:0000CA70       VarTypeIsCustom
 0001:0000CD8C       VarTypeIsValidArrayType
 0001:0000CDB0       VarTypeIsValidElementType
 0001:00009C9C       VarUtils
 0001:00000358       VirtualAlloc
 0001:00000360       VirtualFree
 0001:000055BC       VirtualQuery
 0001:000002EC       VirtualQuery
 0001:000055C4       WaitForSingleObject
 0001:0000323C       WCharFromChar
 0002:000002B8       WesternGroups
 0001:00003DBC       WideCharLenToStrVar
 0001:000002E4       WideCharToMultiByte
 0002:000000C8       Win32BuildNumber
 0001:00008F5C       Win32Check
 0002:000000CC       Win32CSDVersion
 0002:000000C0       Win32MajorVersion
 0002:000000C4       Win32MinorVersion
 0002:000000BC       Win32Platform
 0001:00005664       Windows
 0001:000102CC       WriteCollection
 0001:00015D98       WriteCollectionProp
 0001:00002F84       WriteErrorMessage
 0001:000055CC       WriteFile
 0001:0000022C       WriteFile
 0001:00015FC4       WriteFloatProp
 0001:00016060       WriteInt64Prop
 0001:00016688       WriteInterfaceProp
 0001:00015D2C       WriteIntProp
 0001:0001682C       WriteMethodProp
 0001:00016384       WriteObjectProp
 0001:00015E98       WriteOrdProp
 0001:00015C44       WritePropPath
 0001:00015C98       WriteSet
 0001:00016130       WriteStrProp
 0001:0001696C       WriteVariantProp
 0001:00003764       WStrError
 0001:00003784       WStrSet
 0001:00009E58       _DispInvoke
 0001:00009DC0       _DispInvokeError
 0001:0000B194       _OleVarFromInt
 0001:0000B370       _OleVarFromLStr
 0001:0000B3C0       _OleVarFromPStr
 0001:0000B4BC       _OleVarFromVar
 0001:0000C82C       _SimpleVarNeg
 0001:0000C93C       _SimpleVarNot
 0001:0000BD9C       _SimpleVarOp
 0001:0000C9E4       _VarAddRef
 0001:0000CDE8       _VarArrayGet
 0001:0000CEE0       _VarArrayPut
 0001:0000CC68       _VarArrayRedim
 0001:0000A790       _VarCast
 0001:0000A8AC       _VarCastOle
 0001:00009DE0       _VarClear
 0001:0000C568       _VarCmp
 0001:0000A20C       _VarCopy
 0001:0000C9DC       _VarCopyNoInd
 0001:0000B1E0       _VarFromBool
 0001:0000B238       _VarFromCurr
 0001:0000B330       _VarFromDisp
 0001:0000B35C       _VarFromDynArray
 0001:0000B104       _VarFromInt
 0001:0000B1B4       _VarFromInt64
 0001:0000B304       _VarFromIntf
 0001:0000B250       _VarFromLStr
 0001:0000B27C       _VarFromPStr
 0001:0000B208       _VarFromReal
 0001:0000B220       _VarFromTDateTime
 0001:0000B2CC       _VarFromWStr
 0001:00009DD8       _VarInit
 0001:0000C7E8       _VarNeg
 0001:0000C8F8       _VarNot
 0001:0000A738       _VarOleStrToString
 0001:0000B6AC       _VarOp
 0001:0000A768       _VarStringToOleStr
 0001:0000AB3C       _VarToBool
 0001:0000ACB4       _VarToCurr
 0001:0000B070       _VarToDisp
 0001:0000B0F4       _VarToDynArray
 0001:0000A914       _VarToInt
 0001:0000A9F0       _VarToInt64
 0001:0000AFCC       _VarToIntf
 0001:0000AE28       _VarToLStr
 0001:0000AE9C       _VarToPStr
 0001:0000AB78       _VarToReal
 0001:0000AEEC       _VarToWStr
 0001:0000CB68       _Write0Variant
 0001:0000CAF0       _WriteVariant


  Address         Publics by Value

 0002:FFBE700C       TlsLast
 0001:000001D4       CloseHandle
 0001:000001DC       CreateFileA
 0001:000001E4       GetFileType
 0001:000001EC       GetFileSize
 0001:000001F4       GetStdHandle
 0001:000001FC       RaiseException
 0001:00000204       ReadFile
 0001:0000020C       RtlUnwind
 0001:00000214       SetEndOfFile
 0001:0000021C       SetFilePointer
 0001:00000224       UnhandledExceptionFilter
 0001:0000022C       WriteFile
 0001:00000234       CharNext
 0001:0000023C       ExitProcess
 0001:00000244       MessageBox
 0001:0000024C       FindClose
 0001:00000254       FindFirstFile
 0001:0000025C       FreeLibrary
 0001:00000264       GetCommandLine
 0001:0000026C       GetLastError
 0001:00000274       GetLocaleInfo
 0001:0000027C       GetModuleFileName
 0001:00000284       GetModuleHandle
 0001:0000028C       GetProcAddress
 0001:00000294       GetStartupInfo
 0001:0000029C       GetThreadLocale
 0001:000002A4       LoadLibraryEx
 0001:000002AC       LoadString
 0001:000002B4       lstrcpyn
 0001:000002BC       @strlen
 0001:000002C4       MultiByteToWideChar
 0001:000002CC       RegCloseKey
 0001:000002D4       RegOpenKeyEx
 0001:000002DC       RegQueryValueEx
 0001:000002E4       WideCharToMultiByte
 0001:000002EC       VirtualQuery
 0001:000002F4       SysAllocStringLen
 0001:000002FC       SysReAllocStringLen
 0001:00000304       SysFreeString
 0001:0000030C       InterlockedIncrement
 0001:00000314       InterlockedDecrement
 0001:0000031C       GetCurrentThreadId
 0001:00000324       GetCmdShow
 0001:00000348       LocalAlloc
 0001:00000350       LocalFree
 0001:00000358       VirtualAlloc
 0001:00000360       VirtualFree
 0001:00000368       InitializeCriticalSection
 0001:00000370       EnterCriticalSection
 0001:00000378       LeaveCriticalSection
 0001:00000380       DeleteCriticalSection
 0001:00000388       GetBlockDesc
 0001:000003D8       MakeEmpty
 0001:000003E0       AddBlockAfter
 0001:00000410       DeleteBlock
 0001:00000428       MergeBlockAfter
 0001:0000049C       RemoveBlock
 0001:0000052C       GetSpace
 0001:00000590       GetSpaceAt
 0001:00000608       FreeSpace
 0001:000006C0       Commit
 0001:00000754       Decommit
 0001:000007D4       GetCommitted
 0001:00000864       GetCommittedAt
 0001:00000988       FreeCommitted
 0001:00000A14       InitAllocator
 0001:00000AD8       UninitAllocator
 0001:00000BB8       DeleteFree
 0001:00000C1C       FindCommitted
 0001:00000C4C       FillBeforeGap
 0001:00000C7C       InternalFreeMem
 0001:00000CA0       FillAfterGap
 0001:00000CC8       FillerSizeBeforeGap
 0001:00000D38       FillerSizeAfterGap
 0001:00000D70       DecommitFree
 0001:00000E20       InsertFree
 0001:00000EA8       FreeCurAlloc
 0001:00000EF4       MergeCommit
 0001:00000F80       NewCommit
 0001:00000FAC       NewCommitAt
 0001:00000FE0       SearchSmallBlocks
 0001:0000100C       TryHarder
 0001:00001100       SysGetMem
 0001:00001290       SysFreeMem
 0001:00001434       ResizeInPlace
 0001:00001604       SysReallocMem
 0001:000016C8       @GetMem
 0001:000016E8       @FreeMem
 0001:00001708       @ReallocMem
 0001:00001758       ExceptObject
 0001:00001778       RunErrorAt
 0001:00001784       ErrorAt
 0001:000017D0       Error
 0001:000017DC       @_IOTest
 0001:000017FC       SetInOutRes
 0001:0000180C       IOResult
 0001:0000182C       Move
 0001:0000186C       UpCase
 0001:00001878       @ROUND
 0001:00001884       @AbstractError
 0001:000018A0       OpenText
 0001:000018F8       @RewritText
 0001:00001904       TextIn
 0001:00001940       FileNOPProc
 0001:00001944       TextOut
 0001:00001980       InternalClose
 0001:00001990       TextClose
 0001:000019B0       TextOpen
 0001:00001B5C       InternalFlush
 0001:00001BA4       Flush
 0001:00001BB0       @Flush
 0001:00001BBC       @Close
 0001:00001C14       @AStrCmp
 0001:00001C84       @FillChar
 0001:00001CA4       @ValLong
 0001:00001D70       TryOpenForOutput
 0001:00001DB4       @WriteBytes
 0001:00001E08       @WriteSpaces
 0001:00001E84       @SetEq
 0001:00001E98       FPower10
 0001:00001EA0       @Pow10
 0001:00002180       GetKeyboardType
 0001:00002188       @isNECWindows
 0001:000021B8       @FpuMaskInit
 0001:0000227C       @FpuInit
 0001:00002288       TObject.ClassType
 0001:00002290       TObject.ClassName
 0001:000022A4       TObject.ClassNameIs
 0001:000022CC       TObject.ClassParent
 0001:000022D8       TObject.NewInstance
 0001:000022F4       TObject.FreeInstance
 0001:00002308       TObject.InstanceSize
 0001:00002310       TObject.Create
 0001:00002330       TObject.Destroy
 0001:00002340       TObject.Free
 0001:0000234C       TObject.InitInstance
 0001:000023A4       TObject.CleanupInstance
 0001:000023C4       InvokeImplGetter
 0001:000023F4       TObject.GetInterface
 0001:00002488       TObject.GetInterfaceEntry
 0001:000024CC       @IsClass
 0001:000024F0       GetDynaMethod
 0001:00002520       @CallDynaInst
 0001:00002538       TObject.InheritsFrom
 0001:0000254C       TObject.ClassInfo
 0001:00002554       TObject.SafeCallException
 0001:0000255C       TObject.DefaultHandler
 0001:00002560       TObject.AfterConstruction
 0001:00002564       TObject.BeforeDestruction
 0001:00002568       TObject.Dispatch
 0001:00002590       TObject.MethodAddress
 0001:000025E0       TObject.MethodName
 0001:00002620       TObject.FieldAddress
 0001:00002670       @ClassCreate
 0001:000026C0       @ClassDestroy
 0001:000026C8       @AfterConstruction
 0001:000026D8       @BeforeDestruction
 0001:000026E8       NotifyReRaise
 0001:00002704       NotifyNonDelphiException
 0001:00002728       NotifyExcept
 0001:00002740       NotifyOnExcept
 0001:00002754       NotifyAnyExcept
 0001:00002768       CheckJmp
 0001:00002788       NotifyExceptFinally
 0001:000027B0       NotifyTerminate
 0001:000027CC       NotifyUnhandled
 0001:000027EC       @HandleAnyException
 0001:00002918       @HandleOnException
 0001:00002AA0       @HandleFinally
 0001:00002AD8       @RaiseExcept
 0001:00002B00       @RaiseAgain
 0001:00002B54       @DoneExcept
 0001:00002B84       @TryFinallyExit
 0001:00002B9C       MapToRunError
 0001:00002C3C       @ExceptionHandler
 0001:00002CDC       SetExceptionHandler
 0001:00002CFC       UnsetExceptionHandler
 0001:00002D24       FinalizeUnits
 0001:00002D84       InitUnits
 0001:00002DE4       @StartLib
 0001:00002EAC       @InitResStringImports
 0001:00002ED4       @InitImports
 0001:00002EF8       MakeErrorMessage
 0001:00002F54       ExitDll
 0001:00002F84       WriteErrorMessage
 0001:00003010       @Halt0
 0001:000030E8       @Halt
 0001:000030F4       @RunError
 0001:00003100       @LStrClr
 0001:00003124       @LStrArrayClr
 0001:00003154       @LStrAsg
 0001:00003198       @LStrLAsg
 0001:000031C4       @NewAnsiString
 0001:000031F0       @LStrFromPCharLen
 0001:00003220       CharFromWChar
 0001:0000323C       WCharFromChar
 0001:00003254       @LStrFromPWCharLen
 0001:000032E0       @LStrFromChar
 0001:000032F0       @LStrFromPChar
 0001:00003320       @LStrFromPWChar
 0001:0000335C       @LStrFromString
 0001:00003368       @LStrFromArray
 0001:00003380       @LStrFromWStr
 0001:00003394       @LStrToString
 0001:000033B8       @LStrLen
 0001:000033C0       @LStrCat
 0001:00003404       @LStrCat3
 0001:00003478       @LStrCatN
 0001:000034FC       @LStrCmp
 0001:000035A0       @LStrAddRef
 0001:000035B0       @LStrToPChar
 0001:000035BC       InternalUniqueString
 0001:00003600       UniqueString
 0001:00003608       @UniqueStringA
 0001:00003610       @LStrCopy
 0001:00003650       @LStrDelete
 0001:00003698       @LStrPos
 0001:000036E0       @LStrSetLength
 0001:00003744       @WriteLString
 0001:00003764       WStrError
 0001:0000376C       @NewWideString
 0001:00003784       WStrSet
 0001:00003794       @WStrClr
 0001:000037AC       @WStrArrayClr
 0001:000037D0       @WStrAsg
 0001:000037F4       @WStrFromPCharLen
 0001:00003880       @WStrFromPWCharLen
 0001:000038A4       @WStrFromPWChar
 0001:000038E0       @WStrFromLStr
 0001:000038F0       @WStrToPWChar
 0001:00003900       @WStrLen
 0001:0000390C       @WStrCat
 0001:0000396C       @WStrCmp
 0001:000039F0       @WStrCopy
 0001:00003A3C       @WStrSetLength
 0001:00003A80       @FinalizeRecord
 0001:00003AB4       @FinalizeArray
 0001:00003BA0       @Finalize
 0001:00003BAC       @CopyRecord
 0001:00003CC8       @CopyArray
 0001:00003DBC       WideCharLenToStrVar
 0001:00003DC8       OleStrToStrVar
 0001:00003DEC       StringToOleStr
 0001:00003E10       VariantSystemUndefinedError
 0001:00003E18       VariantSystemDefaultVarClear
 0001:00003E30       InitVariantManager
 0001:00003E50       GetVariantManager
 0001:00003E64       SetVariantManager
 0001:00003E78       @VarClear
 0001:00003E80       @VarCopy
 0001:00003E88       @VarToInt
 0001:00003E90       @VarToInt64
 0001:00003E98       @VarToBool
 0001:00003EA0       @VarToReal
 0001:00003EA8       @VarToCurr
 0001:00003EB0       @VarToLStr
 0001:00003EB8       @VarToWStr
 0001:00003EC0       @VarToIntf
 0001:00003EC8       @VarToDisp
 0001:00003ED0       @VarFromInt
 0001:00003ED8       @VarFromInt64
 0001:00003EEC       @VarFromBool
 0001:00003EF4       @VarFromReal
 0001:00003EFC       @VarFromCurr
 0001:00003F04       @VarFromLStr
 0001:00003F0C       @VarFromWStr
 0001:00003F14       @VarFromIntf
 0001:00003F1C       @VarFromDisp
 0001:00003F24       @VarCmpEQ
 0001:00003F30       @VarClr
 0001:00003F38       @DispCallByIDError
 0001:00003F40       @_llmul
 0001:00003F64       @_lldiv
 0001:00003FE0       @_lludiv
 0001:0000402C       @_llmod
 0001:000040A8       @_llumod
 0001:000040F8       @_llshl
 0001:00004118       @_llushr
 0001:00004138       @ValInt64
 0001:0000435C       @DynArrayLength
 0001:00004364       @DynArrayHigh
 0001:0000436C       CopyArray
 0001:0000437C       FinalizeArray
 0001:00004384       DynArrayClear
 0001:0000438C       DynArraySetLength
 0001:00004518       @DynArraySetLength
 0001:00004524       @DynArrayCopy
 0001:00004544       @DynArrayCopyRange
 0001:00004638       @DynArrayClear
 0001:00004674       @DynArrayAsg
 0001:0000469C       FindHInstance
 0001:000046C4       DelayLoadResourceModule
 0001:0000470C       FindResourceHInstance
 0001:00004734       FindBS
 0001:00004748       ToLongPath
 0001:00004900       LoadResourceModule
 0001:00004B70       AddModuleUnloadProc
 0001:00004B78       RemoveModuleUnloadProc
 0001:00004B80       AddModuleUnloadProc
 0001:00004BA0       RemoveModuleUnloadProc
 0001:00004C00       NotifyModuleUnload
 0001:00004C5C       RegisterModule
 0001:00004C6C       UnregisterModule
 0001:00004CDC       @IntfClear
 0001:00004CF4       @IntfCopy
 0001:00004D20       TInterfacedObject.AfterConstruction
 0001:00004D2C       TInterfacedObject.BeforeDestruction
 0001:00004D3C       TInterfacedObject.NewInstance
 0001:00004D4C       TInterfacedObject.QueryInterface
 0001:00004D74       TInterfacedObject._AddRef
 0001:00004D88       TInterfacedObject._Release
 0001:00004DB0       UnicodeToUtf8
 0001:00004E8C       Utf8ToUnicode
 0001:00004FD0       UTF8Encode
 0001:0000507C       UTF8Decode
 0001:00005120       AnsiToUtf8
 0001:00005170       LoadResString
 0001:000051C8       Finalization
 0001:0000521C       System
 0001:00005290       LocalAlloc
 0001:00005298       LocalFree
 0001:000052A0       TlsAlloc
 0001:000052A8       TlsFree
 0001:000052B0       TlsGetValue
 0001:000052B8       TlsSetValue
 0001:000052C0       AllocTlsBuffer
 0001:000052CC       GetTlsSize
 0001:000052D4       InitThreadTLS
 0001:00005318       InitProcessTLS
 0001:00005344       ExitThreadTLS
 0001:0000536C       ExitProcessTLS
 0001:00005390       @GetTls
 0001:000053D0       InitializeModule
 0001:000053DC       @InitLib
 0001:00005424       Finalization
 0001:00005454       SysInit
 0001:0000545C       Finalization
 0001:0000548C       Types
 0001:00005494       CloseHandle
 0001:0000549C       CompareString
 0001:000054A4       CreateEvent
 0001:000054AC       CreateFile
 0001:000054B4       DeleteCriticalSection
 0001:000054BC       EnterCriticalSection
 0001:000054C4       EnumCalendarInfoA
 0001:000054CC       FormatMessage
 0001:000054D4       GetACP
 0001:000054DC       GetCPInfo
 0001:000054E4       GetCurrentThreadId
 0001:000054EC       GetDiskFreeSpaceA
 0001:000054F4       GetLastError
 0001:000054FC       GetLocaleInfo
 0001:00005504       GetModuleFileName
 0001:0000550C       GetModuleHandle
 0001:00005514       GetProcAddress
 0001:0000551C       GetStdHandle
 0001:00005524       GetStringTypeEx
 0001:0000552C       GetSystemDirectory
 0001:00005534       GetThreadLocale
 0001:0000553C       GetTickCount
 0001:00005544       GetVersionEx
 0001:0000554C       GetWindowsDirectory
 0001:00005554       GlobalAlloc
 0001:0000555C       GlobalFree
 0001:00005564       GlobalLock
 0001:0000556C       GlobalHandle
 0001:00005574       GlobalReAlloc
 0001:0000557C       GlobalUnlock
 0001:00005584       InitializeCriticalSection
 0001:0000558C       LeaveCriticalSection
 0001:00005594       ReadFile
 0001:0000559C       ResetEvent
 0001:000055A4       SetEndOfFile
 0001:000055AC       SetEvent
 0001:000055B4       SetFilePointer
 0001:000055BC       VirtualQuery
 0001:000055C4       WaitForSingleObject
 0001:000055CC       WriteFile
 0001:000055D4       CharNext
 0001:000055DC       GetSystemMetrics
 0001:000055E4       LoadString
 0001:000055EC       MessageBox
 0001:000055F4       GlobalAllocPtr
 0001:00005604       GlobalReAllocPtr
 0001:00005620       GlobalFreePtr
 0001:00005634       Finalization
 0001:00005664       Windows
 0001:0000566C       Finalization
 0001:0000569C       Messages
 0001:00005934       Finalization
 0001:00005964       SysConst
 0001:00006508       ConvertErrorFmt
 0001:0000652C       AllocMem
 0001:0000654C       LowerCase
 0001:00006588       CompareMem
 0001:000065A8       CompareText
 0001:000065FC       SameText
 0001:00006620       AnsiCompareStr
 0001:00006658       AnsiCompareText
 0001:00006690       IsValidIdent
 0001:000066F4       IntToStr
 0001:00006724       IntToStr
 0001:00006758       StrToInt
 0001:00006794       StrToIntDef
 0001:000067AC       StrToInt64
 0001:00006808       FileOpen
 0001:00006864       FileCreate
 0001:00006888       FileCreate
 0001:00006890       FileRead
 0001:000068BC       FileWrite
 0001:000068E8       FileSeek
 0001:00006920       FileClose
 0001:00006928       LastDelimiter
 0001:00006978       ExtractFileName
 0001:000069B0       BackfillGetDiskFreeSpaceEx
 0001:00006A24       StrLen
 0001:00006A3C       StrMove
 0001:00006A4C       StrLCopy
 0001:00006A80       StrComp
 0001:00006AA4       StrLIComp
 0001:00006AE8       StrScan
 0001:00006B08       StrPos
 0001:00006B5C       StrPas
 0001:00006B70       StrAlloc
 0001:00006B84       StrNew
 0001:00006BB0       FormatError
 0001:00006C08       FormatVarToStr
 0001:00006C1C       FormatClearStr
 0001:00006C28       FormatBuf
 0001:0000703C       StrLFmt
 0001:0000707C       Format
 0001:00007090       FmtStr
 0001:00007150       PutExponent
 0001:00007194       FloatToText
 0001:0000746C       FloatToDecimal
 0001:00007698       SysErrorMessage
 0001:000076E4       GetLocaleStr
 0001:00007730       GetLocaleChar
 0001:00007758       LocalGetLocaleStr
 0001:00007794       GetMonthDayNames
 0001:000078B8       EnumEraNames
 0001:000078F4       EnumEraYearOffsets
 0001:0000796C       GetEraNamesAndYearOffsets
 0001:00007A1C       TranslateDateFormat
 0001:00007C44       ConvertAddr
 0001:00007C50       ExceptionErrorMessage
 0001:00007DD8       ShowException
 0001:00007E8C       Exception.Create
 0001:00007EC8       Exception.CreateFmt
 0001:00007F48       Exception.CreateRes
 0001:00007F84       Exception.CreateResFmt
 0001:00008018       EHeapException.FreeInstance
 0001:00008044       CreateInOutError
 0001:000080C4       ErrorHandler
 0001:00008118       CreateAssertException
 0001:000081C4       RaiseAssertException
 0001:000081D4       AssertErrorHandler
 0001:000081F0       AbstractErrorHandler
 0001:00008208       MapException
 0001:00008288       GetExceptionClass
 0001:000082A0       CreateAVObject
 0001:0000846C       GetExceptionObject
 0001:00008538       ExceptHandler
 0001:00008548       InitExceptions
 0001:000085CC       DoneExceptions
 0001:00008638       InitPlatformId
 0001:00008690       ByteTypeTest
 0001:00008708       ByteType
 0001:0000872C       StrByteType
 0001:00008744       StrCharLength
 0001:00008764       CharLength
 0001:000087A0       AnsiPos
 0001:000087D8       AnsiStrPos
 0001:00008878       AnsiStrRScan
 0001:000088A0       AnsiStrScan
 0001:000088E0       LCIDToCodePage
 0001:00008954       InitLeadBytes
 0001:000089B4       IsWesternGroup
 0001:000089CC       InitSysLocale
 0001:00008B40       GetFormatSettings
 0001:00008EB8       Sleep
 0001:00008EC0       RaiseLastOSError
 0001:00008F5C       Win32Check
 0001:00008F6C       FreeTerminateProcs
 0001:00008F8C       InitDriveSpacePtr
 0001:00008FE8       InterlockedIncrement
 0001:00008FF4       InterlockedDecrement
 0001:00009000       InterlockedExchange
 0001:00009008       InterlockedExchangeAdd
 0001:00009010       TThreadLocalCounter.Create
 0001:0000904C       TThreadLocalCounter.Destroy
 0001:000090B4       TThreadLocalCounter.HashIndex
 0001:000090CC       TThreadLocalCounter.Open
 0001:00009144       TThreadLocalCounter.Close
 0001:000091CC       TThreadLocalCounter.Delete
 0001:00009214       TThreadLocalCounter.Reattach
 0001:00009240       TThreadLocalCounter.Recycle
 0001:00009298       TMultiReadExclusiveWriteSynchronizer.Create
 0001:0000930C       TMultiReadExclusiveWriteSynchronizer.Destroy
 0001:00009354       TMultiReadExclusiveWriteSynchronizer.BlockReaders
 0001:00009360       TMultiReadExclusiveWriteSynchronizer.UnblockReaders
 0001:0000936C       TMultiReadExclusiveWriteSynchronizer.UnblockOneWriter
 0001:00009378       TMultiReadExclusiveWriteSynchronizer.WaitForReadSignal
 0001:00009388       TMultiReadExclusiveWriteSynchronizer.WaitForWriteSignal
 0001:00009398       TMultiReadExclusiveWriteSynchronizer.BeginWrite
 0001:00009498       TMultiReadExclusiveWriteSynchronizer.EndWrite
 0001:0000953C       TMultiReadExclusiveWriteSynchronizer.BeginRead
 0001:000095E0       TMultiReadExclusiveWriteSynchronizer.EndRead
 0001:00009670       FreeAndNil
 0001:00009680       Supports
 0001:000096A4       Supports
 0001:00009A0C       Finalization
 0001:00009B8C       SysUtils
 0001:00009C0C       VariantInit
 0001:00009C14       VariantClear
 0001:00009C1C       VariantCopy
 0001:00009C24       VariantCopyInd
 0001:00009C2C       VariantChangeTypeEx
 0001:00009C34       SafeArrayCreate
 0001:00009C3C       SafeArrayRedim
 0001:00009C44       SafeArrayGetLBound
 0001:00009C4C       SafeArrayGetUBound
 0001:00009C54       SafeArrayGetElement
 0001:00009C5C       SafeArrayPutElement
 0001:00009C64       SafeArrayPtrOfIndex
 0001:00009C6C       Finalization
 0001:00009C9C       VarUtils
 0001:00009DC0       _DispInvokeError
 0001:00009DC8       VarCastError
 0001:00009DD0       VarInvalidOp
 0001:00009DD8       _VarInit
 0001:00009DE0       _VarClear
 0001:00009E58       _DispInvoke
 0001:00009EC4       Increment
 0001:00009F20       VarArrayCopyForEach
 0001:0000A0E0       VarArrayCopyProc
 0001:0000A0F4       VarCopyCommon
 0001:0000A20C       _VarCopy
 0001:0000A214       VarCopyNoInd
 0001:0000A21C       VarInt64FromVar
 0001:0000A3B8       VarInt64ToVar
 0001:0000A530       AnyChangeType
 0001:0000A598       ChangeSourceAny
 0001:0000A5B0       VarChangeType
 0001:0000A738       _VarOleStrToString
 0001:0000A768       _VarStringToOleStr
 0001:0000A788       VarStringToOleStr
 0001:0000A790       _VarCast
 0001:0000A8AC       _VarCastOle
 0001:0000A914       _VarToInt
 0001:0000A9F0       _VarToInt64
 0001:0000AB3C       _VarToBool
 0001:0000AB78       _VarToReal
 0001:0000ACB4       _VarToCurr
 0001:0000AE28       _VarToLStr
 0001:0000AE9C       _VarToPStr
 0001:0000AEEC       _VarToWStr
 0001:0000AF5C       AnyToIntf
 0001:0000AFCC       _VarToIntf
 0001:0000B070       _VarToDisp
 0001:0000B0F4       _VarToDynArray
 0001:0000B104       _VarFromInt
 0001:0000B194       _OleVarFromInt
 0001:0000B1B4       _VarFromInt64
 0001:0000B1E0       _VarFromBool
 0001:0000B208       _VarFromReal
 0001:0000B220       _VarFromTDateTime
 0001:0000B238       _VarFromCurr
 0001:0000B250       _VarFromLStr
 0001:0000B27C       _VarFromPStr
 0001:0000B2CC       _VarFromWStr
 0001:0000B304       _VarFromIntf
 0001:0000B330       _VarFromDisp
 0001:0000B35C       _VarFromDynArray
 0001:0000B370       _OleVarFromLStr
 0001:0000B3C0       _OleVarFromPStr
 0001:0000B410       OleVarFromAny
 0001:0000B474       OleVarFromVarArrayProc
 0001:0000B4BC       _OleVarFromVar
 0001:0000B5F8       VarStrCat
 0001:0000B6AC       _VarOp
 0001:0000B924       Failure
 0001:0000B928       AnyOp
 0001:0000B9B4       CheckType
 0001:0000B9FC       RealOp
 0001:0000BA8C       IntOp
 0001:0000BBB0       Int64Op
 0001:0000BD9C       _SimpleVarOp
 0001:0000C1B4       VarCompare
 0001:0000C568       _VarCmp
 0001:0000C570       CheckType
 0001:0000C594       IntCompare
 0001:0000C5A8       Int64Compare
 0001:0000C5E4       RealCompare
 0001:0000C60C       StringCompare
 0001:0000C684       SimpleVarCmp
 0001:0000C7E8       _VarNeg
 0001:0000C82C       _SimpleVarNeg
 0001:0000C8F8       _VarNot
 0001:0000C93C       _SimpleVarNot
 0001:0000C9DC       _VarCopyNoInd
 0001:0000C9E4       _VarAddRef
 0001:0000CA08       VarType
 0001:0000CA0C       VarIsClear
 0001:0000CA70       VarTypeIsCustom
 0001:0000CA9C       VarSameValue
 0001:0000CAE0       SetClearVarToEmptyParam
 0001:0000CAF0       _WriteVariant
 0001:0000CB68       _Write0Variant
 0001:0000CB70       GetVarDataArrayInfo
 0001:0000CBBC       VarArrayCreate
 0001:0000CC68       _VarArrayRedim
 0001:0000CCBC       GetVarArray
 0001:0000CCE4       VarArrayDimCount
 0001:0000CD0C       VarArrayLowBound
 0001:0000CD34       VarArrayHighBound
 0001:0000CD5C       VarIsArray
 0001:0000CD64       VarIsArray
 0001:0000CD8C       VarTypeIsValidArrayType
 0001:0000CDB0       VarTypeIsValidElementType
 0001:0000CDE8       _VarArrayGet
 0001:0000CEBC       VarArrayGet
 0001:0000CEE0       _VarArrayPut
 0001:0000D028       VarArrayPut
 0001:0000D050       DynArrayIndex
 0001:0000D090       DynArrayElTypeInfo
 0001:0000D0AC       DynArrayDim
 0001:0000D0C4       DynArraySize
 0001:0000D0CC       IsDynArrayRectangular
 0001:0000D134       DynArrayBounds
 0001:0000D188       DecIndices
 0001:0000D1F4       DynArrayVariantBounds
 0001:0000D24C       DynArrayVarType
 0001:0000D274       DynArrayToVariant
 0001:0000D588       DynArrayFromVariant
 0001:0000D864       ClearVariantTypeList
 0001:0000D8D4       TCustomVariantType.BinaryOp
 0001:0000D8E0       TCustomVariantType.Cast
 0001:0000D918       TCustomVariantType.CastTo
 0001:0000D960       TCustomVariantType.Compare
 0001:0000D96C       TCustomVariantType.CompareOp
 0001:0000D9A4       TCustomVariantType.CastToOle
 0001:0000D9E0       TCustomVariantType.Destroy
 0001:0000DA64       TCustomVariantType.IsClear
 0001:0000DA68       TCustomVariantType.LeftPromotion
 0001:0000DA7C       TCustomVariantType.OlePromotion
 0001:0000DA84       TCustomVariantType.RaiseCastError
 0001:0000DA8C       TCustomVariantType.RaiseInvalidOp
 0001:0000DA94       TCustomVariantType.RaiseDispError
 0001:0000DA9C       TCustomVariantType.RightPromotion
 0001:0000DAB0       TCustomVariantType.UnaryOp
 0001:0000DAB8       TCustomVariantType.DispInvoke
 0001:0000DAC4       TCustomVariantType._AddRef
 0001:0000DAD0       TCustomVariantType._Release
 0001:0000DADC       TCustomVariantType.QueryInterface
 0001:0000DB04       FindCustomVariantType
 0001:0000DBA4       FindCustomVariantType
 0001:0000DC8C       Null
 0001:0000DCA0       Finalization
 0001:0000DD04       Variants
 0001:0000DFB8       Finalization
 0001:0000DFE8       RTLConsts
 0001:0000E01C       GetTypeData
 0001:0000E028       GetEnumName
 0001:0000E11C       GetEnumNameValue
 0001:0000E168       GetEnumValue
 0001:0000E1CC       GetPropInfo
 0001:0000E23C       GetPropInfos
 0001:0000E290       IsStoredProp
 0001:0000E2C0       GetOrdProp
 0001:0000E334       SetOrdProp
 0001:0000E390       GetShortStrProp
 0001:0000E3D4       SetShortStrProp
 0001:0000E428       GetShortStrPropAsLongStr
 0001:0000E450       SetShortStrPropAsLongStr
 0001:0000E484       AssignLongStr
 0001:0000E498       GetLongStrProp
 0001:0000E4D8       SetLongStrProp
 0001:0000E518       GetWideStrPropAsLongStr
 0001:0000E570       SetWideStrPropAsLongStr
 0001:0000E5C8       GetStrProp
 0001:0000E608       SetStrProp
 0001:0000E634       GetWideStrProp
 0001:0000E71C       SetWideStrProp
 0001:0000E7F0       GetFloatProp
 0001:0000E908       SetFloatProp
 0001:0000EB00       AssignVariant
 0001:0000EB14       GetVariantProp
 0001:0000EB54       SetVariantProp
 0001:0000EB94       GetMethodProp
 0001:0000EBD4       SetMethodProp
 0001:0000EC0C       GetInt64Prop
 0001:0000EC34       SetInt64Prop
 0001:0000EC70       GetInterfaceProp
 0001:0000ECF0       SetInterfaceProp
 0001:0000ED64       Finalization
 0001:0000EDB4       TypInfo
 0001:0000EDBC       Finalization
 0001:0000EDEC       ActiveX
 0001:0000FCB8       TRegGroup.Create
 0001:0000FD34       TRegGroup.Destroy
 0001:0000FD74       TRegGroup.GetClass
 0001:0000FDD4       PointerInModule
 0001:0000FDF4       TRegGroup.UnregisterModuleClasses
 0001:0000FE98       TRegGroups.Create
 0001:0000FF0C       TRegGroups.Destroy
 0001:0000FF68       TRegGroups.GetClass
 0001:0000FFAC       TRegGroups.Lock
 0001:0000FFB8       TRegGroups.Unlock
 0001:0000FFC4       TRegGroups.UnregisterModuleClasses
 0001:0000FFF4       TClassFinder.GetClass
 0001:0001007C       GetFieldClassTable
 0001:00010088       ClassNotFound
 0001:000100F4       GetClass
 0001:00010148       UnRegisterModuleClasses
 0001:00010194       FindIntToIdent
 0001:00010210       FindIdentToInt
 0001:0001028C       FindGlobalComponent
 0001:000102CC       WriteCollection
 0001:00010338       CollectionsEqual
 0001:0001045C       TList.Destroy
 0001:0001047C       TList.Add
 0001:000104B0       TList.Clear
 0001:000104C8       TList.Delete
 0001:00010528       ReturnAddr
 0001:0001052C       TList.Error
 0001:00010564       TList.Error
 0001:000105B8       TList.Get
 0001:000105E0       TList.Grow
 0001:00010614       TList.IndexOf
 0001:00010634       TList.Last
 0001:00010640       TList.Put
 0001:00010694       TList.Remove
 0001:000106B4       TList.SetCapacity
 0001:000106F0       TList.SetCount
 0001:00010760       TList.Notify
 0001:00010764       TThreadList.Create
 0001:000107B8       TThreadList.Destroy
 0001:00010834       TThreadList.Add
 0001:000108BC       TThreadList.LockList
 0001:000108D0       TThreadList.UnlockList
 0001:000108DC       TPersistent.Destroy
 0001:00010908       TPersistent.Assign
 0001:0001091C       TPersistent.AssignError
 0001:000109EC       TPersistent.AssignTo
 0001:000109F4       TPersistent.DefineProperties
 0001:000109F8       TPersistent.GetNamePath
 0001:00010AA8       TPersistent.GetOwner
 0001:00010AAC       GetDesigner
 0001:00010B44       NotifyDesigner
 0001:00010BA8       TCollection.Destroy
 0001:00010BF4       TCollection.Add
 0001:00010C00       TCollection.Assign
 0001:00010C98       TCollection.BeginUpdate
 0001:00010C9C       TCollection.Changed
 0001:00010CAC       TCollection.Clear
 0001:00010D14       TCollection.EndUpdate
 0001:00010D20       TCollection.GetAttrCount
 0001:00010D24       TCollection.GetAttr
 0001:00010D30       TCollection.GetItemAttr
 0001:00010D50       TCollection.GetCount
 0001:00010D58       TCollection.GetItem
 0001:00010D6C       TCollection.GetNamePath
 0001:00010E34       TCollection.GetPropName
 0001:00010F50       TCollection.SetItemName
 0001:00010F54       TCollection.Update
 0001:00010F58       TCollection.Added
 0001:00010F5C       TCollection.Deleting
 0001:00010F60       TCollection.Notify
 0001:00010F84       TStrings.Destroy
 0001:00010FB4       TStrings.Add
 0001:00010FD8       TStrings.AddObject
 0001:00010FFC       TStrings.AddStrings
 0001:000110B4       TStrings.Assign
 0001:00011144       TStrings.BeginUpdate
 0001:0001115C       DoWrite
 0001:000111B4       TStrings.DefineProperties
 0001:00011200       TStrings.EndUpdate
 0001:00011214       TStrings.Equals
 0001:000112BC       ReturnAddr
 0001:000112C0       TStrings.Error
 0001:000112F8       TStrings.Error
 0001:00011350       TStrings.Exchange
 0001:00011438       TStrings.GetCapacity
 0001:00011440       TStrings.GetObject
 0001:00011444       TStrings.GetText
 0001:00011498       TStrings.GetTextStr
 0001:000115C0       TStrings.IndexOf
 0001:0001164C       TStrings.IndexOfName
 0001:00011714       TStrings.IndexOfObject
 0001:00011748       TStrings.InsertObject
 0001:00011778       TStrings.LoadFromFile
 0001:000117CC       TStrings.LoadFromStream
 0001:00011878       TStrings.Move
 0001:00011928       TStrings.Put
 0001:00011958       TStrings.PutObject
 0001:0001195C       TStrings.ReadData
 0001:00011A0C       TStrings.SaveToFile
 0001:00011A64       TStrings.SaveToStream
 0001:00011AC0       TStrings.SetCapacity
 0001:00011AC4       TStrings.SetStringsAdapter
 0001:00011AF8       TStrings.SetText
 0001:00011B48       TStrings.SetTextStr
 0001:00011C08       TStrings.SetUpdateState
 0001:00011C0C       TStrings.WriteData
 0001:00011C90       TStrings.CompareStrings
 0001:00011C9C       TStringList.Destroy
 0001:00011CF8       TStringList.Add
 0001:00011D04       TStringList.AddObject
 0001:00011D68       TStringList.Changed
 0001:00011D84       TStringList.Changing
 0001:00011DA0       TStringList.Clear
 0001:00011DE0       TStringList.Delete
 0001:00011E4C       TStringList.Exchange
 0001:00011EA8       TStringList.ExchangeItems
 0001:00011ECC       TStringList.Find
 0001:00011F44       TStringList.Get
 0001:00011F78       TStringList.GetCapacity
 0001:00011F7C       TStringList.GetCount
 0001:00011F80       TStringList.GetObject
 0001:00011FA8       TStringList.Grow
 0001:00011FDC       TStringList.IndexOf
 0001:00012018       TStringList.Insert
 0001:00012028       TStringList.InsertObject
 0001:0001207C       TStringList.InsertItem
 0001:000120F4       TStringList.Put
 0001:00012150       TStringList.PutObject
 0001:00012190       TStringList.QuickSort
 0001:00012224       TStringList.SetCapacity
 0001:00012240       TStringList.SetUpdateState
 0001:00012258       StringListCompareStrings
 0001:0001226C       TStringList.Sort
 0001:0001227C       TStringList.CustomSort
 0001:000122B4       TStringList.CompareStrings
 0001:000122D0       TStream.GetPosition
 0001:000122F0       TStream.SetPosition
 0001:00012304       TStream.GetSize
 0001:00012350       TStream.SetSize
 0001:00012354       TStream.SetSize64
 0001:00012368       TStream.SetSize
 0001:000123BC       RaiseException
 0001:00012408       TStream.Seek
 0001:0001248C       TStream.Seek
 0001:000124FC       TStream.WriteBuffer
 0001:00012534       TStream.WriteDescendent
 0001:00012590       THandleStream.Create
 0001:000125CC       THandleStream.Read
 0001:000125DC       THandleStream.Write
 0001:000125EC       THandleStream.Seek
 0001:00012618       THandleStream.SetSize
 0001:0001262C       THandleStream.SetSize
 0001:00012654       TFileStream.Create
 0001:00012698       TFileStream.Create
 0001:00012760       TFileStream.Destroy
 0001:00012794       TCustomMemoryStream.SetPointer
 0001:0001279C       TCustomMemoryStream.Read
 0001:000127D4       TCustomMemoryStream.Seek
 0001:000127F8       TMemoryStream.Destroy
 0001:00012824       TMemoryStream.Clear
 0001:0001283C       TMemoryStream.SetCapacity
 0001:00012864       TMemoryStream.SetSize
 0001:00012890       TMemoryStream.Realloc
 0001:0001291C       TMemoryStream.Write
 0001:0001296C       TFiler.Create
 0001:000129B4       TFiler.Destroy
 0001:000129DC       TFiler.SetRoot
 0001:00012AB8       TPropFixup.Create
 0001:00012B10       TPropFixup.MakeGlobalReference
 0001:00012B58       TPropFixup.ResolveReference
 0001:00012B68       TPropIntfFixup.ResolveReference
 0001:00012BEC       FindNestedComponent
 0001:00012CB4       RemoveFixupReferences
 0001:00012D60       RemoveFixups
 0001:00012DE4       ReadError
 0001:00012DFC       PropValueError
 0001:00012E08       PropertyNotFound
 0001:00012E34       TReader.Destroy
 0001:00012E70       TReader.CheckValue
 0001:00012E94       TReader.DefineProperty
 0001:00012EC8       TReader.DefineBinaryProperty
 0001:00012FA4       TReader.EndOfList
 0001:00012FB8       TReader.Error
 0001:00012FD8       TReader.FindMethod
 0001:00013040       RemoveGlobalFixup
 0001:000130BC       TReader.DoFixupReferences
 0001:000131DC       TReader.FlushBuffer
 0001:00013200       TReader.FreeFixups
 0001:0001323C       TReader.GetFieldClass
 0001:000132D0       TReader.GetPosition
 0001:000132E8       TReader.NextValue
 0001:000132F8       TReader.PropertyError
 0001:0001330C       TReader.Read
 0001:00013358       TReader.ReadBuffer
 0001:00013394       TReader.ReadChar
 0001:000133EC       TReader.ReadCollection
 0001:00013498       ComponentCreated
 0001:000134B8       Recover
 0001:00013518       CreateComponent
 0001:00013628       SetCompName
 0001:000136C8       FindExistingComponent
 0001:0001376C       TReader.ReadComponent
 0001:00013944       TReader.ReadData
 0001:000139B4       TReader.ReadDataInner
 0001:00013A84       TReader.ReadFloat
 0001:00013AC4       TReader.ReadSingle
 0001:00013B04       TReader.ReadCurrency
 0001:00013B50       TReader.ReadDate
 0001:00013B90       TReader.ReadIdent
 0001:00013C90       TReader.ReadInteger
 0001:00013CFC       TReader.ReadInt64
 0001:00013D40       TReader.ReadListBegin
 0001:00013D48       TReader.ReadListEnd
 0001:00013D50       TReader.ReadPrefix
 0001:00013D90       HandleException
 0001:00013E90       PropPathError
 0001:00013EAC       TReader.ReadProperty
 0001:0001408C       SetIntIdent
 0001:000140D4       SetObjectIdent
 0001:00014114       SetInterfaceReference
 0001:000141D4       TReader.ReadPropValue
 0001:000144F8       TReader.ReadSet
 0001:000145B4       TReader.ReadStr
 0001:000145F0       TReader.ReadString
 0001:000146AC       TReader.ReadWideString
 0001:00014790       TReader.ReadValue
 0001:000147A4       TReader.SkipSetBody
 0001:000147EC       SkipList
 0001:00014814       SkipBinary
 0001:00014844       SkipCollection
 0001:000148A0       TReader.SkipValue
 0001:00014A3C       TReader.SkipProperty
 0001:00014A84       TReader.SkipComponent
 0001:00014B2C       TReader.FindAncestorComponent
 0001:00014BE4       TReader.ReferenceName
 0001:00014BFC       TReader.SetName
 0001:00014C24       TReader.FindComponentClass
 0001:00014C98       TReader.SkipBytes
 0001:00014CE0       ReadCustomVariant
 0001:00014EA0       TReader.ReadVariant
 0001:00015098       TWriter.Destroy
 0001:000150C4       TWriter.AddAncestor
 0001:000150D0       TWriter.DefineProperty
 0001:000150F8       TWriter.DefineBinaryProperty
 0001:00015124       TWriter.GetPosition
 0001:00015134       TWriter.FlushBuffer
 0001:0001513C       TWriter.SetPosition
 0001:00015178       TWriter.SetRoot
 0001:00015190       TWriter.Write
 0001:000151DC       TWriter.WriteBinary
 0001:00015264       TWriter.WriteBuffer
 0001:0001527C       TWriter.WriteChar
 0001:000152CC       TWriter.WriteCollection
 0001:0001536C       FindAncestor
 0001:000153BC       TWriter.WriteComponent
 0001:00015498       TWriter.WriteData
 0001:00015898       TWriter.WriteDescendent
 0001:000158C0       TWriter.WriteFloat
 0001:000158E4       TWriter.WriteSingle
 0001:00015908       TWriter.WriteCurrency
 0001:0001592C       TWriter.WriteDate
 0001:00015950       TWriter.WriteIdent
 0001:00015A14       TWriter.WriteInteger
 0001:00015A88       TWriter.WriteInteger
 0001:00015AE0       TWriter.WriteListBegin
 0001:00015AE8       TWriter.WriteListEnd
 0001:00015AF0       TWriter.WritePrefix
 0001:00015B34       TWriter.WriteProperties
 0001:00015BFC       AncestorValid
 0001:00015C44       WritePropPath
 0001:00015C98       WriteSet
 0001:00015D2C       WriteIntProp
 0001:00015D98       WriteCollectionProp
 0001:00015E3C       IsDefaultValue
 0001:00015E98       WriteOrdProp
 0001:00015F6C       IsDefaultValue
 0001:00015FC4       WriteFloatProp
 0001:00016010       IsDefaultValue
 0001:00016060       WriteInt64Prop
 0001:000160A8       IsDefault
 0001:00016130       WriteStrProp
 0001:0001619C       OwnedBy
 0001:000161B4       GetComponentValue
 0001:000162DC       ObjectAncestorMatch
 0001:00016324       IsDefault
 0001:00016384       WriteObjectProp
 0001:000165B4       IsDefaultValue
 0001:00016688       WriteInterfaceProp
 0001:000167A8       IsDefaultValue
 0001:0001682C       WriteMethodProp
 0001:000168E0       IsDefaultValue
 0001:0001696C       WriteVariantProp
 0001:000169DC       TWriter.WriteProperty
 0001:00016AF4       TWriter.WriteVariant
 0001:00016EEC       TWriter.WritePropName
 0001:00016F40       TWriter.WriteSignature
 0001:00016F50       TWriter.WriteStr
 0001:00016F98       TWriter.WriteMinStr
 0001:00017030       TWriter.WriteString
 0001:00017084       TWriter.WriteWideString
 0001:00017138       TWriter.WriteValue
 0001:0001714C       TComponent.Create
 0001:00017198       TComponent.Destroy
 0001:00017210       TComponent.BeforeDestruction
 0001:0001721C       TComponent.ReadLeft
 0001:00017230       TComponent.ReadTop
 0001:00017244       TComponent.WriteLeft
 0001:00017250       TComponent.WriteTop
 0001:0001725C       TComponent.Insert
 0001:00017288       TComponent.Remove
 0001:000172B0       TComponent.InsertComponent
 0001:00017308       TComponent.RemoveComponent
 0001:00017340       TComponent.DestroyComponents
 0001:00017398       TComponent.Destroying
 0001:000173D4       TComponent.RemoveNotification
 0001:000173F8       TComponent.RemoveFreeNotification
 0001:00017414       TComponent.Notification
 0001:00017470       TComponent.DefineProperties
 0001:000174F8       TComponent.HasParent
 0001:000174FC       TComponent.GetChildren
 0001:00017504       TComponent.GetChildOwner
 0001:00017508       TComponent.GetChildParent
 0001:0001750C       TComponent.GetNamePath
 0001:00017520       TComponent.GetOwner
 0001:00017524       TComponent.SetChildOrder
 0001:00017528       TComponent.GetParentComponent
 0001:0001752C       TComponent.SetParentComponent
 0001:00017530       TComponent.Updating
 0001:0001753C       TComponent.Updated
 0001:00017548       TComponent.Loaded
 0001:00017554       TComponent.PaletteCreated
 0001:00017558       TComponent.ReadState
 0001:00017560       TComponent.WriteState
 0001:00017568       TComponent.ValidateRename
 0001:000175E8       TComponent.ValidateContainer
 0001:000175FC       TComponent.ValidateInsert
 0001:00017600       TComponent.FindComponent
 0001:00017650       TComponent.SetName
 0001:000176DC       TComponent.ChangeName
 0001:000176F0       TComponent.GetComponent
 0001:0001771C       TComponent.GetComponentCount
 0001:0001772C       TComponent.SetDesigning
 0001:0001777C       TComponent.SetReference
 0001:000177C4       TComponent.ExecuteAction
 0001:000177EC       TComponent.UpdateAction
 0001:00017814       TComponent.SafeCallException
 0001:0001782C       TComponent.UpdateRegistry
 0001:00017834       TComponent.QueryInterface
 0001:00017874       TComponent._AddRef
 0001:00017894       TComponent._Release
 0001:000178B4       TComponent.IntfGetComponent
 0001:000178B8       FreeIntConstList
 0001:00017924       ModuleUnload
 0001:0001792C       Finalization
 0001:000179D4       Classes
 0001:00017A38       MsgBox
 0001:00017B2C       GetWinDir
 0001:00017BA4       GetSysDir
 0001:00017C34       StrToStrList
 0001:00017CFC       Eng
 0001:00017F48       Finalization
 0001:00017FE8       pluginexample
 0002:00000000       ExitCode
 0002:00000004       ErrorAddr
 0002:00000008       FileMode
 0002:0000000C       Default8087CW
 0002:00000010       HeapAllocFlags
 0002:00000014       DebugHook
 0002:00000018       JITEnable
 0002:0000001C       NoErrMsg
 0002:00000020       DefaultTextLineBreakStyle
 0002:00000024       LibModuleList
 0002:00000028       ModuleUnloadList
 0002:0000002C       MemoryManager
 0002:00000038       reMap
 0002:00000054       runErrMsg
 0002:00000074       errCaption
 0002:0000007C       dig
 0002:0000008C       Module
 0002:000000A4       TlsProc
 0002:000000B4       EmptyStr
 0002:000000B8       EmptyWideStr
 0002:000000BC       Win32Platform
 0002:000000C0       Win32MajorVersion
 0002:000000C4       Win32MinorVersion
 0002:000000C8       Win32BuildNumber
 0002:000000CC       Win32CSDVersion
 0002:000000D0       LeadBytes
 0002:000000F0       HexDisplayPrefix
 0002:000000F4       GetDiskFreeSpaceEx
 0002:000000F8       cSimpleBoolStrs
 0002:00000100       AccessMode
 0002:0000010C       ShareMode
 0002:00000120       FormatErrorStrs
 0002:00000128       FCon1E18
 0002:00000134       DCon10
 0002:00000138       DefShortMonthNames
 0002:00000168       DefLongMonthNames
 0002:00000198       DefShortDayNames
 0002:000001B4       DefLongDayNames
 0002:000001D0       ErrorMap
 0002:00000208       ExceptMap
 0002:000002B8       WesternGroups
 0002:000002BC       TerminateProcList
 0002:000002C0       CVarTypeToElementInfo
 0002:000003C8       BaseTypeMap
 0002:000003E0       OpTypeMap
 0002:00000434       CInvalidCustomVariantType
 0002:00000438       CBooleanToRelationship
 0002:00000444       CRelationshipToBoolean
 0002:00000458       BooleanIdents
 0002:00000460       DotSep
 0002:00000464       FilerSignature
 0002:00000468       NilMethod
 0002:00000470       ValTypeToVarType
 0002:0000049C       SyncList
 0002:00001000       DispCallByIDProc
 0002:00001004       ExceptProc
 0002:00001008       ErrorProc
 0002:0000100C       ExceptClsProc
 0002:00001010       ExceptObjProc
 0002:00001014       RaiseExceptionProc
 0002:00001018       RTLUnwindProc
 0002:0000101C       ExceptionClass
 0002:00001020       AssertErrorProc
 0002:00001024       ExitProcessProc
 0002:00001028       AbstractErrorProc
 0002:0000102C       MainInstance
 0002:00001030       MainThreadID
 0002:00001034       IsLibrary
 0002:00001038       CmdShow
 0002:0000103C       CmdLine
 0002:00001040       ExitProc
 0002:00001044       IsConsole
 0002:00001045       IsMultiThread
 0002:00001046       Test8086
 0002:00001048       Input
 0002:00001214       Output
 0002:000013E0       ErrOutput
 0002:000015AC       AllocMemCount
 0002:000015B0       AllocMemSize
 0002:000015B4       .5
 0002:000015B8       initialized
 0002:000015BC       heapErrorCode
 0002:000015C0       heapLock
 0002:000015D8       blockDescBlockList
 0002:000015DC       blockDescFreeList
 0002:000015E0       spaceRoot
 0002:000015F0       decommittedRoot
 0002:00001600       avail
 0002:0000160C       rover
 0002:00001610       remBytes
 0002:00001614       curAlloc
 0002:00001618       smallTab
 0002:0000161C       committedRoot
 0002:0000162C       InitContext
 0002:00001658       VariantManager
 0002:00001704       ModuleIsLib
 0002:00001705       ModuleIsCpp
 0002:00001708       TlsIndex
 0002:00001710       HInstance
 0002:00001714       DllProc
 0002:00001718       .1
 0002:0000171C       tlsBuffer
 0002:00001720       .1
 0002:00001724       .3
 0002:00001728       .1
 0002:0000172C       .1
 0002:00001730       CurrencyString
 0002:00001734       CurrencyFormat
 0002:00001735       NegCurrFormat
 0002:00001736       ThousandSeparator
 0002:00001737       DecimalSeparator
 0002:00001738       CurrencyDecimals
 0002:00001739       DateSeparator
 0002:0000173C       ShortDateFormat
 0002:00001740       LongDateFormat
 0002:00001744       TimeSeparator
 0002:00001748       TimeAMString
 0002:0000174C       TimePMString
 0002:00001750       ShortTimeFormat
 0002:00001754       LongTimeFormat
 0002:00001758       ShortMonthNames
 0002:00001788       LongMonthNames
 0002:000017B8       ShortDayNames
 0002:000017D4       LongDayNames
 0002:000017F0       SysLocale
 0002:000017FE       ListSeparator
 0002:00001800       EraNames
 0002:0000181C       EraYearOffsets
 0002:00001838       TrueBoolStrs
 0002:0000183C       FalseBoolStrs
 0002:00001840       .94
 0002:00001844       OutOfMemory
 0002:00001848       InvalidPointer
 0002:0000184C       FLanguages
 0002:00001850       .1
 0002:00001854       EmptyParam
 0002:00001864       VarDispProc
 0002:00001868       ClearAnyProc
 0002:0000186C       ChangeAnyProc
 0002:00001870       RefAnyProc
 0002:00001874       .3
 0002:00001878       GVariantManager
 0002:00001924       GOldVariantManager
 0002:000019D0       LVarTypes
 0002:000019D4       LVarTypeSync
 0002:000019D8       .1
 0002:000019DC       .6
 0002:000019E0       .3
 0002:000019E4       GlobalNameSpace
 0002:000019E8       .35
 0002:000019EC       IntConstList
 0002:000019F0       RegGroups
 0002:000019F4       FindGlobalComponentProcs
 0002:000019F8       GlobalFixupList
 0002:000019FC       ThreadLock
    42 0001:00017A38
    45 0001:00017A64    46 0001:00017A72    47 0001:00017A79    48 0001:00017A80
    49 0001:00017A87    50 0001:00017A8E    53 0001:00017A93    54 0001:00017AB7
    55 0001:00017ABB    56 0001:00017AC2    57 0001:00017AC9    58 0001:00017AD0
    59 0001:00017AD7    62 0001:00017AD9    63 0001:00017AE3    65 0001:00017AEB
    66 0001:00017B21    72 0001:00017B2C    73 0001:00017B4B    74 0001:00017B5C
    75 0001:00017B6A    76 0001:00017B75    77 0001:00017B9C    83 0001:00017BA4
    84 0001:00017BC3    85 0001:00017BD4    86 0001:00017BE7    88 0001:00017BF2
    89 0001:00017BFE    91 0001:00017C07    92 0001:00017C2E   100 0001:00017C34
   101 0001:00017C67   104 0001:00017C70   105 0001:00017C7D   106 0001:00017C8C
   108 0001:00017CAA   102 0001:00017CC5   110 0001:00017CF3   122 0001:00017CFC
   123 0001:00017D1E   125 0001:00017D2C   129 0001:00017D36   131 0001:00017D45
   134 0001:00017D55   136 0001:00017D7C   139 0001:00017D8F   140 0001:00017DB6
   143 0001:00017DC9   146 0001:00017DF0   147 0001:00017E54   154 0001:00017E5C
   155 0001:00017E73   158 0001:00017E88   159 0001:00017E90   161 0001:00017EC5
   166 0001:00017FE8   168 0001:00017FF8

Bound resource files

pluginexample.drf


Program entry point at 0001:00017FE8
